:1000000028C400005EC400005CC400005AC40000A4
:1000100058C4000056C4000054C4000052C400007C
:1000200050C400004EC400000C94D6300C94BE3175
:100030000C948B3046C4000044C4000042C400004D
:1000400040C400003EC400003CC400003AC40000AC
:1000500038C400000C94B23034C4000032C4000034
:1000600030C400002EC400002CC400002AC40000CC
:1000700028C4000026C4000024C4000022C40000DC
:1000800020C400001EC400001CC400001AC40000EC
:1000900018C4000016C4000014C4000012C40000FC
:1000A00010C400000EC400000CC4000005010902C9
:1000B000A10185020901A1000509190129081500FE
:1000C0002501950875018102050109300931158165
:1000D000257F95027508810609381581257F9501D0
:1000E00075088106050C0A38021581257F95017572
:1000F000088106C0C005010980A101850319012AF4
:10010000B700150126B700950175108100C0050CD8
:100110000901A101850419012AA002150126A002E6
:10012000950175108100C005010906A1018506052C
:100130000719E029E71500250195087501810205D9
:1001400007190029EF1500250195F07501810205B9
:10015000081901290595057501910295017503910D
:1001600001C00660FF0961A1010962150026FF00B8
:100170009520750881020963150026FF00952075FA
:10018000089102C005010906A101050719E029E748
:1001900015002501950875018102950175088101F9
:1001A0000507190029FF150026FF0095067508812F
:1001B000000508190129051500250195057501910E
:1001C00002950175039101C00000000000000000CD
:1001D000000000000000000000000000000000001F
:1001E0000000000000000000000000007E0F00D4AE
:1001F000FFFFFFC7000000780000000000000000C3
:100200002A2B280000000000000000000000000071
:1002100000000029000000002C1E3420212224347C
:100220002627252E362D3738271E1F20212223244E
:1002300025263333362E37381F0405060708090AEA
:100240000B0C0D0E0F101112131415161718191A86
:100250001B1C1D2F3130232D350405060708090A04
:100260000B0C0D0E0F101112131415161718191A66
:100270001B1C1D2F3130354C09025B00030100A00F
:10028000FA09040000010301010009211101000124
:10029000224400070581030800010904010002034C
:1002A000000000092111010001222200070582033C
:1002B00020000107050303200001090402000103D7
:1002C00000000009211101000122B6000705840386
:1002D0002000011201000200000008544D0220011C
:1002E00000010203011C037600690061006C003A02
:1002F00000660036003400630032006200330063A1
:100300000000000E034E00430052002D0038003064
:1003100000000006034D00540000000403090429F6
:100320000000003A003B003C003D003E003F004022
:100330000035001E001F00200021002200230024A1
:100340000025002B0014001A000800150017001CDF
:100350000018000C00390004001600070009000A0C
:10036000000B000D000E00E10000001D001B000648
:10037000001900050011001000E0000000E200E498
:1003800000000000002C00E600000000000000005B
:100390000045004400430000004200410027004B9C
:1003A000004A002A0000002E0049002D002600000F
:1003B000004E004D00310030002F004C00130012A1
:1003C000000000000052002800000034000000334C
:1003D000000F0000004F0051000000E50038005001
:1003E000003700360001000000010001000100019B
:1003F00000010001000100010001000100010001F5
:1004000000010001000100010001000100010001E4
:1004100000010001000100010001000100010001D4
:1004200000010001000100010001000100010000C5
:1004300000010001000100010001000100010001B4
:1004400000000001000100000000000100010000A8
:1004500000000000000000007C010001000000011D
:100460000001000100010001000100000001000185
:100470000001000100000001000100010001000175
:100480000001000100010000000000010001000067
:100490000001000000010001000000010001000057
:1004A000000100010001000100010022232526288F
:1004B000292A2C2D2F3032333536383A3B3D3E40F9
:1004C00042434547494A4C4E5051535557595A5C3F
:1004D0005E6062646668696B6D6F71737577797B56
:1004E0007D7F81838587898A8C8E90929496989A55
:1004F0009C9E9FA1A3A5A7A8AAACAEAFB1B3B4B66A
:10050000B8B9BBBCBEBFC1C2C3C5C6C7C9CACBCCC4
:10051000CDCED0D1D2D2D3D4D5D6D7D7D8D9D9DA97
:10052000DADBDBDBDCDCDCDCDCDDDDDDDDDCDCDC0C
:10053000DCDCDBDBDBDADAD9D9D8D7D7D6D5D4D334
:10054000D2D2D1D0CECDCCCBCAC9C7C6C5C3C2C109
:10055000BFBEBCBBB9B8B6B4B3B1AFAEACAAA8A766
:10056000A5A3A19F9E9C9A98969492908E8C8A891E
:10057000878583817F7D7B79777573716F6D6B69FB
:1005800068666462605E5C5A5957555351504E4CD0
:100590004A4947454342403E3D3B3A38363533327F
:1005A000302F2D2C2A292826252322FFAA7F5540CB
:1005B0000001010101010101010102020202020226
:1005C00002020203030303030303030404040404F9
:1005D00004040505050505060606060607070707C0
:1005E0000708080808090909090A0A0A0B0B0B0C75
:1005F0000C0C0D0D0D0E0E0E0F0F0F101011111112
:100600001212131314141515161617171818191992
:100610001A1A1B1B1C1D1D1E1E1F202021222223F7
:100620002424252626272829292A2B2C2D2D2E2F38
:1006300030313232333435363738393A3B3C3D3E4F
:100640003F404142434445464748494A4C4D4E4F3E
:1006500050515354555658595A5B5D5E5F61626400
:10066000656668696B6C6D6F7072737577787A7B8D
:100670007D7E8082838587888A8C8E8F91939596E4
:10068000989A9C9EA0A2A3A5A7A9ABADAFB1B3B504
:10069000B7BABCBEC0C2C4C6C9CBCDCFD1D4D6D8E0
:1006A000DBDDDFE2E4E7E9EBEEF0F3F5F8FAFDFF7E
:1006B0001E0F0500047F3F1F643214643214783C1F
:1006C0001E1E140A05FD377A585A000004E6D6B4F7
:1006D000460200210116000000742FE5A3E0035735
:1006E000014A5D003D8889C65436C3174FE4E32FA5
:1006F00092B5A85075CFC8C9E98BEB7E10F7A5F469
:100700001FE7F0E8EB3194B2077FA2B41184E61E34
:100710006FD53F5564DEF023E89A5446EA4513B09E
:1007200038B2AB092728D06A6746FC10367C44F300
:10073000115223B9397BBB303D6296429F0A152086
:1007400080C04C41E0097F0349DDA118DC1821C2BB
:100750006C3782892673B65960134AF7FC9CAAEE5F
:1007600084A39F5938F3BCDE2A92E0BCADA24F208F
:10077000B8C23434EEAF069B4DA7B234CD4347DC4C
:10078000F4F186561B63AFD6570C1AC1A94B4663CA
:10079000962F5BFE48DD3728C7BB854E18BAFFFF92
:1007A000BD7D12F7F3B923A55D878D5291063266A0
:1007B00099B1A20027BB6171944B90A68A770B6B0D
:1007C00047CE184DCDB541B394B22544A1C6E14BF7
:1007D000FF9301688E3B8D2757437D47397FA3E008
:1007E0009AB0C63AC41BA7029BF4BEB433CAD071F8
:1007F0007BF12BA88D7D986AB8D135BACF4EF4C85D
:10080000446333A0763797DDC8787F02653081A6D0
:1008100077A171CF48DA670C4684EFFCA82F9CDAE9
:100820007113BFA81E8C033A6813E5491800000035
:10083000007139B00744EBB4D50001E602D80600D8
:1008400000E692E59EB1C467FB0200000000045977
:100850005A0011241FBECFEFDAE0DEBFCDBF04B6D1
:1008600003FE18C08091F5069091F606A091F70658
:10087000B091F8068730904BA740B04B59F41092D6
:10088000F5061092F6061092F7061092F806E0E0D0
:10089000F8E3099526E0A6EEB1E001C01D92A53F60
:1008A000B207E1F711E0A0E0B1E0E2E2F9E602C050
:1008B00005900D92A63EB107D9F70E94BD280C9471
:1008C00011349ECB9C019A9581159F4118F5F32F09
:1008D000F270EE27832F8170732F74706627532F69
:1008E0005870442734FF0CC08295807FEF2B09F0AD
:1008F0008062672B09F08064452B69F08068089559
:10090000EF2B09F08260672B09F08460452B19F00A
:100910008860089580E00895CF93DF93EB01D2DFE4
:10092000FE010995DF91CF910895982F92959F70C0
:1009300024E0911102C020E0982F892F869586959A
:10094000811511F02E5F982F892F8695820F0895BB
:10095000982F909580FD08C02D9A91FF07C0469A68
:1009600092FF06C0479A08952D98F7CF4698F8CF82
:10097000479808958093AA0608958093AB0608953A
:1009800021E030E001C0220F8A95EAF78091AB06A2
:10099000822BF3CF21E030E0A90102C0440F551FA4
:1009A0008A95E2F7CA0180959091AB068923E5CF3D
:1009B000292F9B3090F5893080F590E039E0239F16
:1009C000800D911D1124282F277041E001C0440F94
:1009D0002A95EAF723E0969587952A95E1F7FC0199
:1009E000EE0FFF1FE80FF91FED5AFA4F20E030E03D
:1009F00070E05191DF01CB01022E02C096958795E0
:100A00000A94E2F7817081958527842385278E9348
:100A10002F5F3F4F2330310561F70895292F9B3019
:100A200078F5893068F590E039E0239F800D911DBD
:100A30001124682F677023E0969587952A95E1F732
:100A4000FC01EE0FFF1FE80FF91FED5AFA4F40E0CF
:100A500050E080E0219130E0062E02C036952795C7
:100A60000A94E2F721703327042E01C0220F0A9462
:100A7000EAF7822B4F5F5F4F4330510559F70895D6
:100A800080E008959091AB0621E030E0F90101C0CB
:100A9000EE0F8A95EAF7D90102C0AA0FBB1F6A952B
:100AA000E2F7EA2B01C0220F4A95EAF7892F8E233D
:100AB000E81303C0892F822B60CF2095822F8923D2
:100AC000FBCF8091B3069091B206981301C00895B0
:100AD0008F5F8770FACF9091AD06809589238093C0
:100AE000AD06282F2770211110C0891771F0909141
:100AF000F40692FF0AC08695869586954BDF109284
:100B0000AD061092AF061092AE0608959091A80619
:100B1000982B9093A8060895982F90958091A806F9
:100B200089238093A80608958091A706811531F046
:100B30001092A7061092B1061092B0060895803E5A
:100B40009105D9F1C8F48133910509F482C048F4C4
:100B50008932910509F472C08A32910509F480C086
:100B6000089589339105E9F082389105D1F08533F4
:100B7000910509F45EC00895843E9105D9F148F4C9
:100B8000823E910539F1833E910549F181EE90E075
:100B90000895863E9105C9F1873E910509F43EC04E
:100BA00008952091F3062370211164C02091F4066A
:100BB00023FF14C089E290E008952091F30620FD00
:100BC00045C03091F40630FF09C024FD24C083EEF7
:100BD00090E008952091F30622FDF7CF089520912B
:100BE000F30622FD44C03091F40630FD43C024FFDB
:100BF000F5CF11C02091F40621FFF0CF8091F306CC
:100C000084FD09C087EE90E008952091F30623FF4C
:100C1000E5CF24FFF7CF80E090E008952091F30620
:100C200023FD2BC03091F40631FFE1CF84EE90E03C
:100C300008952091F30625FFD1CFBCCF2091F30674
:100C400025FD1EC02091F40623FFC8CF89E390E064
:100C500008952091F30626FFC1CF8AE290E008951F
:100C60002091F30626FFBACF81E390E0089582EE4B
:100C700090E0089580EE90E0089586EE90E008956B
:100C800085E390E008959091F30692FF10C041E053
:100C9000282F2471243009F040E031E0282F2871FA
:100CA000283009F030E0431711F02CE0822793FF41
:100CB00010C041E0282F2471243109F040E031E0D8
:100CC000282F2871283109F030E0431711F02CE06B
:100CD00082273091F40630FF10C051E0282F217197
:100CE000213009F050E041E0282F2871283009F028
:100CF00040E0541711F029E0822731FF10C041E095
:100D0000282F2171213109F040E031E0282F28718E
:100D1000283109F030E0431711F029E0822794FDD3
:100D2000877E08951F93CF93DF9309DFEC01811530
:100D300022E5920708F052C0811540E5940708F0BB
:100D4000CDC0803E910520F58D3C910508F0A1C0F5
:100D5000883A910570F4853A910508F097C0813082
:100D60009105B9F10497813A910598F1C0E0D0E07E
:100D700030C0885A91094B97C8F7C85AD0E0CC0FB9
:100D8000DD1FC758DE4F0990D881C02DD46421C023
:100D9000811550E49507B0F4C11580E2D80708F03A
:100DA000B3C0C83ED105A8F0CE019A9581159F41E8
:100DB000E8F68D2F68DF182FCE019927C0DEEC01F1
:100DC000D12B07C09927BBDECC27DF70C82BD92BCE
:100DD000D06ACE01DF91CF911F910895803842E50E
:100DE0009407C8F5803652E5950708F05BC0C0341B
:100DF00082E5D807D0F4C03292E5D90708F04BC09D
:100E00008C2F8695869520E2829FC0011124C370A5
:100E100021E030E0A90102C0440F551FCA95E2F756
:100E2000EA01C82BD92BDD68D4CF8C2F8695869507
:100E3000877050E2859FC0011124C37021E030E02B
:100E4000A90102C0440F551FCA95E2F7EA01C82B59
:100E5000D92BDC68BECF803C52E5950758F48F71E2
:100E6000C03AD245A0F590E0982F8827EC01C46FD6
:100E7000D06AAFCF805C9245809708F077CFDC2FA7
:100E8000CC27CC27DF71C06FD06AA3CFA497D064E2
:100E9000A0CFD0659ECFCF71D0E0DC2FCC27C16F23
:100EA000D06A97CF86958695877020E2829FC00191
:100EB0001124C37021E030E0A90102C0440F551F86
:100EC000CA95E2F7EA01C82BD92BDA6882CFDBDEBC
:100ED000C82FD0E0DC2FCC27D0627BCF8F71D3DE40
:100EE00093E0CC0FDD1F9A95E1F7CC27DF70282F18
:100EF00030E084FF05C050E1859F90011124332725
:100F0000C22BD32BD06965CF8D2F8F71BCDE182FEC
:100F1000CE01992714DEEC01D12BDECF80E00895BD
:100F2000F894E82FE295EF70F0E041A18F7021E096
:100F300030E0B90102C0660F771F8A95E2F7CB0156
:100F4000962F9095942391A392A1892B82A37894B4
:100F500008950895CF92DF92EF92FF921F93CF935F
:100F6000DF93172FE82FF0E0E055FA4F71110CC016
:100F7000E4918E2F7E2F6E2FDF91CF911F91FF90E6
:100F8000EF90DF90CF900895E62EF12CC72ED12C54
:100F9000F491EF2F86E0689F90011124CFEFD0E00D
:100FA000C901BE010E942232AB01EE0CFF1C65E5B7
:100FB000649FC001659F900D1124E81AF90A6E2DF7
:100FC000660F6E0D7E01EC18FD08FE9DD001FF9DA1
:100FD000B00D11248B2F169F70011124EF2CFF24CC
:100FE0006E01CE18DF087601FE9D6001FF9DD00CDA
:100FF00011247E01E61AF108B701169F7001179FB0
:10100000F00C1124EF2CFF24CE19DF09FC9F700196
:10101000FD9FF00C11247F2D43305105C1F02C3F72
:10102000334058F441305105B1F04230510509F0D8
:10103000A2CFEB2F8F2D7F2F9ECF4430510571F023
:101040004630510509F497CF7B2F8D2D94CF7D2D00
:10105000EB2F8F2F90CF7F2FED2D8DCFEF2D7B2F6F
:10106000F8CFCF93982F762F842FC22F692F72DF5E
:10107000472F282F8C2F90E04AD2CF91089580914E
:101080009E06843060F48370846080939E06809115
:10109000A106853B18F084EB8093A10608958C3A55
:1010A000B0F38370886AF1CFCF93DF9380919E066F
:1010B00080FD0BC0C0E0D0E020E040E060E0CE0169
:1010C00026D22196C135D105B9F7B1D6DF91CF919E
:1010D0000895FF920F931F93CF93DF93182F062F3E
:1010E000F42E80919E0680FF0CC0C0E0D0E02F2D32
:1010F000402F612FCE010BD22196C135D105B9F712
:10110000D3DFCDB7DEB7E5E00C948B32CF93DF931E
:10111000EC012091A1069C81892F817090FD822F86
:10112000692F627091FD622F492F447092FD422F0A
:10113000D0DF8C8190E00196877099278C83DF91B6
:10114000CF910895982F762F842F20919E0620FF0F
:101150000AC0453B08F084EB692FFCDE962F672F11
:10116000482F892FB6CF0895CF93DF93EC01EEE996
:10117000F6E0438162818C81E5DF8C818F5F8C8317
:10118000DF91CF910895CF93DF93EC01EC81F0E0F4
:10119000E555FB4F4491EEE9F6E062818181D2DFB3
:1011A0008C818F5F8C83DF91CF9108950F931F9374
:1011B000CF93DF93EC0100E010E04091A106453BA6
:1011C00008F044EB802F880F800F9C81980160917C
:1011D000A006890F46DF0F5F1F4F0135110569F724
:1011E00063DF8C819A8190FF07C08F5F8C83DF91D2
:1011F000CF911F910F9108958150F8CFEF92FF92F8
:101200000F931F93CF93DF93FC018281FF24F3940C
:1012100080FF02C0FF24FA94C0E0D0E020E040E06C
:1012200060E0CE0174D104E010E0E12C8091C204B2
:101230008E0D8235A4F161E50E941532892F082EAA
:10124000001C00088C170D0691F44091A1060403C0
:10125000A00111245595479555954795453B08F0B4
:1012600044EB9E016091A00680919F06FADEEF0C90
:1012700001501040D9F62196C135D10579F614DF19
:101280008091C204F1E0FF120EC0811591F08150EF
:101290008093C204CDB7DEB7E6E00C948A3287FFB4
:1012A000CECF8F5ACCCF90E00196BE010E9436324D
:1012B000EFCF80E5EDCFCF93DF93C0E0D0E020E02B
:1012C00040E060E0CE0123D12196C135D105B9F7C8
:1012D000C0E0D0E08091C104082E001C0008C817AF
:1012E000D00574F180910601082E001C00088C17AF
:1012F0000D0634F14091A106453B08F044EB9E01F8
:101300006091A00680919F06ACDE2196C135D10583
:1013100009F7CADE809105019091C104980F90935E
:10132000C10420910601280F20930601121614F41F
:1013300090351CF0819580930501DF91CF91089540
:1013400020E040E060E0CE01E2D0DFCFA6E0B0E0F8
:10135000ECEAF9E00C946C328D839E83AD81BE8102
:101360001496FC912F2F30E0D9010E9402349B018A
:10137000AC010E94D0336B017C0180E290E09C01C3
:101380002F1B3109F901A5E5B0E0A70196010E94E4
:10139000D03369837A838B839C839F01DF010E9412
:1013A00056329B010E945C329B01AC012C0D3D1D0D
:1013B0004E1D5F1D69817A818B819C810E94E03383
:1013C000022F30E00A32B8F5C901880F991F820F49
:1013D000931F95958795182F1095E12CF12C85E595
:1013E000D82ED01A8D2DE1FC802F412F153B08F00F
:1013F00044EB97016091A00634DE5FEFE51AF50A31
:1014000081E5E816F10471F74FDEAD81BE811496D7
:101410009C9181E0911519F0903219F48FEF80932F
:10142000040180910401890FED81FE818483269659
:10143000E8E00C94883285E590E0AC01421B530B48
:101440009A01CA01880F991F820F931F97FFC1CF7E
:101450000196BFCF0F931F93CF93DF93EC0120E052
:1014600030E06091A00680919F069C8189010F5F0A
:101470001F4F2832310554F4911501F14091A10616
:10148000453B08F044EBEDDD9801EBCF911116C020
:101490004091A106453B08F044EBE3DD980101359E
:1014A0001105F9F601DE8C8190E001968170992793
:1014B0008C83DF91CF911F910F91089540E0EDCF84
:1014C00081152CE7920741F42091200530912105E8
:1014D000232B11F480E090E00895E6E1F6E080E04F
:1014E00090E060E876E243EA56E225E137E277836E
:1014F000668351874087338722879787868701963F
:1015000070968830910599F708956A9A0895FC01BC
:10151000EE0FFF1FE80FF91FE05DFD4F6183408371
:1015200022830895FC018481862381110AC082816F
:101530008115B9F06823908593FF05C081E06111A2
:101540000FC080E00895282F22952F708F70282BD0
:10155000962F92959F706F70962B81E02913F1CF93
:10156000089581E008950F931F93CF9301E010E059
:10157000082E01C0000F0A94EAF7C091A6069C2F1E
:101580009023911115C09091AD06969596959695DC
:10159000891306C01092AD061092AF061092AE06E7
:1015A000EFD9C027C093A606CF911F910F91089540
:1015B000F1D9F7CF282F35EB2303C001112497FF72
:1015C00004C080589109892F089580589F4FFBCF00
:1015D00080917C0580FD14C081FD14C082FD16C081
:1015E00080917B05811581F08E3180F420E5829F0A
:1015F000C00111246EE170E00E943632862F0895FA
:1016000084E1089588E2089588E0089580E50895CA
:1016100080917C0580FD17C081FD17C082FD19C037
:1016200080917A05811599F0883298F428E0829F9C
:10163000C001112468E270E00E9436326115710524
:1016400051F0862F089562E0FCCF64E0FACF61E0AC
:10165000F8CF68E0F6CF81E00895FA01309709F0FD
:1016600009950895E0914905F0914A05309739F0C0
:101670000190F081E02D309711F00995089580E0F8
:101680000895A3E0B0E0E7E4FBE00C9472329C0123
:1016900080912E0290912F0282179307B1F0309320
:1016A0002F0220932E02E0914905F0914A053097D0
:1016B00061F00084F185E02D309739F083E0898373
:1016C0003B832A83CE01019609952396E2E00C9490
:1016D0008E32A3E0B0E0EFE6FBE00C9472329C01A6
:1016E00080912C0290912D0282179307B1F03093D4
:1016F0002D0220932C02E0914905F0914A05309784
:1017000061F00084F185E02D309739F084E0898321
:101710003B832A83CE01019609952396E2E00C943F
:101720008E3290912001913091F0AAEEB1E0EFEF6E
:1017300090E02D91821751F0EF3F19F4211101C073
:10174000E92F9F5F9630A9F7EF3FC9F40895909174
:10175000F30697FFEACFE82FE695E695E695803FFA
:10176000A8F7F0E0E051FE4F877021E030E001C0C3
:10177000220F8A95EAF78281822B828308950E2EAA
:10178000000CFF0BE851FE4FF8CF909120019130F3
:1017900021F49091F30697FD0CC0EAEEF1E09191EF
:1017A000891302C0DF011E9251E0E03FF507B9F74F
:1017B0000895E82FE695E695E695803FC8F7F0E0B6
:1017C000E051FE4F877021E030E0A90102C0440FD4
:1017D000551F8A95E2F7CA018095928189238283F9
:1017E000089580911F0108952FB7F89480912802E1
:1017F00090912902A0912A02B0912B022FBF089547
:10180000CF93DF93C091A8068091AC06C82B80913E
:10181000A7068115F1F0E8DF2091B0063091B106FE
:10182000821B930B8838934108F07ED9D091A7068C
:1018300080912001813021F48091F30687FD13C04F
:1018400086E02AEE31E090E0815088F491116CD965
:10185000CD2B8091920580958C2390919105892BB9
:10186000DF91CF9108958EE122EF31E0ECCFF901C5
:1018700041919F01411541F39F5FE6CF962F209143
:10188000F40622FF0EC0682F660F660F660F692BE5
:101890006093AD0675D8A8DF9093AF068093AE062F
:1018A00008956EC89091A706292F2823211559F075
:1018B000809589238093A706811531F095DF809369
:1018C000B0069093B106089580E090E0F8CF8CDFE9
:1018D00020917F0530918005232B211521F08093E5
:1018E0000305909304052091810530918205232BF7
:1018F000211521F08093010590930205E09149059F
:10190000F0914A05309759F00680F781E02D309725
:1019100031F082E080937D058DE795E0099508958B
:10192000611509F441C0E3E3E80FE33148F4F0E066
:10193000ED5EFB4C0C9449324BDE81958093800523
:10194000C6CF46DEFBCF44DE819580937F05F8CF7E
:101950003FDEFBCF5DDE80938105F2CF59DE8195BE
:10196000FACF56DE819580938205EACF51DEFBCF18
:10197000815D990B21E030E001C0220F8A95EAF7E2
:1019800080917E05822B80937E05DACF80917C0545
:10199000816080937C05D4CF80917C058260F9CFF3
:1019A00080917C058460F5CF40917F058D3C59F492
:1019B0008091800587FF0DC010928005411559F474
:1019C00010927B0508C08E3C81F48091800518162A
:1019D0009CF3411581F08091810590918205892BBE
:1019E0008111AECF10927A05ABCF8F3C41F447FF07
:1019F000F0CF10927F05809180058115E0CF803D6A
:101A000019F41416B4F3E5CF90918105893D29F4BA
:101A10001916FCF610928105DCCF8A3D19F497FF68
:101A2000D8CFF8CF909182058B3D29F497FFD1CF85
:101A300010928205CECF8C3D19F41916CCF3C9CF84
:101A40009FE2980F983090F4815D990B21E030E08F
:101A5000B90102C0660F771F8A95E2F7CB01809526
:101A600090917E05892380937E05B3CF8D3D31F41F
:101A700080917C058E7F80937C05ABCF8E3D21F4D9
:101A800080917C058D7FF7CF8F3D09F0A2CF8091AB
:101A90007C058B7FF0CF2FB7F8946091280270916E
:101AA000290280912A0290912B022FBF0895CF9294
:101AB000DF92EF92FF92CF93DF93D82FC92FC09080
:101AC0001006D0901106E0901206F0901306E3DFA6
:101AD0006C197D098E099F09643F7140810591054C
:101AE00010F1D9DF6B017C0182E390E0A0E0B0E06F
:101AF000C092F704D092F804E092F904F092FA044C
:101B00008093F3049093F404A093F504B093F60447
:101B1000D0930E06C0930F06DF91CF91FF90EF9008
:101B2000DF90CF90089584EF91E0A0E0B0E0E0CFA7
:101B3000FC019B0180911E0290911F02861797075E
:101B400040F0672B29F48091E8008E778093E800BD
:101B5000C90140E0009741F4411106C08091E800BE
:101B600082FF2FC080E00895209122052115A9F160
:101B70002530A9F12091E80023FD2DC02091E80037
:101B800022FDECCF2091E80020FFE4CF3091F3005C
:101B90002091F200009719F02830310558F041E00B
:101BA0002830310509F040E02091E8002E7720939D
:101BB000E800D0CF41914093F10001972F5F3F4F54
:101BC000E9CF80912205811541F0853041F0809167
:101BD000E80083FFC3CF81E0089582E0089583E0A9
:101BE00008958091180287FF13C08091E80082FF5A
:101BF00006C08091E8008B778093E800089580917B
:101C000022058111F2CF0895809122058115D9F323
:101C10008091E80080FFF8CF8091E8008E77ECCFCC
:101C20002091E4003091E50095E6A9012091EC00B7
:101C3000822F817020FF06C08091E80080FF06C0DF
:101C400080E008952091E80022FD1AC080912205CD
:101C5000811589F0853089F08091EB0085FD0FC0FA
:101C60002091E4003091E50042175307F9F29A956C
:101C7000E1F684E0089582E0089583E0089581E02C
:101C80000895E8EDF0E080818E7F80831092E2007D
:101C90001092DA001092E100A0EEB0E08C91816029
:101CA0008C9380818F77808319BCA7EDB0E08C91F5
:101CB0008E7F8C9380818F7E80831092170208958F
:101CC000E0914905F0914A05309739F00284F38597
:101CD000E02D309711F060E209950895982F9093C8
:101CE000E900891771F07091EC002091ED0050919E
:101CF000F00021FD09C09F5F973089F78093E900CC
:101D00000895762F242F50E03091EB003E7F3093E2
:101D1000EB003091ED003D7F3093ED003091EB0012
:101D200031603093EB007093EC002093ED00509302
:101D3000F0002091EE0027FDDECF0895A0E0B0E096
:101D4000E4EAFEE00C946C32C8EDD0E088818F7E2E
:101D50008883E7EDF0E080818160808384E082BF4A
:101D600081E08093170288818E7F888302EE10E0E5
:101D7000F80110821092DA0081EEC82ED12CF60103
:101D8000108288818F7788838881806888838881A2
:101D90008F7D888319BC1092220510921602109232
:101DA000DB041092150290EEE92EF12CF7018081F0
:101DB0008B7F808388818160888342E060E080E05F
:101DC0008DDFF60180818E7F8083F80180818160C4
:101DD0008083808188608083F70180818E7F80830B
:101DE000888180618883CDB7DEB7E8E00C948832C3
:101DF000E091B3069091B20627E0E91302C080E0BB
:101E00000895AE2FB0E02E9FF0011124EC54F94F4D
:101E10003181361306C03081381303C03581341345
:101E200004C0FD013196E770E8CF81E008953EB12E
:101E30003B7F2EB124604FB7F89480E392E0FC0121
:101E40000196508168E02EB9000000C057FF3EB9EE
:101E5000550F000000C000C000C03EB900C06A9528
:101E600091F753E08332950751F74FBF8FE594E028
:101E70000197F1F700C00000089581E08093E00031
:101E800080E28093D8001092C9008FE19EE4019710
:101E9000F1F700C0000087E090EBDC018093F506CD
:101EA0009093F606A093F706B093F80688E19CE0BD
:101EB0000FB6F894A895809360000FBE90936000D1
:101EC000FFCF0F931F93CF93DF938B01EA01909184
:101ED0002205943051F58093E9008FEF9091E8004E
:101EE00095FD06C095ED9A95F1F700008A95B1F73A
:101EF0008091E80085FF19C093DE811111C08091A7
:101F0000E80085FD06C08091E8008E778093E800A8
:101F1000F3CFF80181918F018093F100219779F738
:101F20008091E8008E778093E800DF91CF911F9138
:101F30000F910895792F603229F440E250E0682F24
:101F400082E0BFCF0895CF93DF93D82FC92F48E009
:101F500050E0682F792F81E0B4DF88E0ED2FFC2F6F
:101F6000A0E2B2E001900D928A95E1F7DF91CF9166
:101F70000895BC0140E250E084E0A3CFBC0146E0FC
:101F800050E084E09ECFBC0143E050E084E099CF74
:101F90009091F40692FB222720F9281779F080FB14
:101FA00092F99093F4066091F3067091F40684E040
:101FB00090E00E94993382E00C946B0508951F9382
:101FC000CF93DF93962F122F632F8330D8F49B305B
:101FD000C8F44930B8F4C42FD0E0CC0FDD1F22E1A3
:101FE000929FC00DD11D112496EC899FC00DD11D6B
:101FF0001124CE0189960E947F33612FCE018A96EB
:102000000E947F33DF91CF911F910895809120012D
:10201000813061F58091F30687FF28C0F1DB809362
:10202000F10140E250E069E275E080EF91E00E944A
:102030003A33892BD1F080E2E0EFF1E0A9E2B5E09C
:1020400001900D928A95E1F7E0914905F0914A05DA
:10205000309759F00480F581E02D309731F086E01B
:102060008093F00180EF91E009950895C9DB80939A
:10207000E80148E050E06BE475E088EE91E00E94F2
:102080003A33892B91F388E0E8EEF1E0ABE4B5E078
:1020900001900D928A95E1F7E0914905F0914A058A
:1020A000309719F30280F381E02D3097F1F288EE3A
:1020B00091E0DACF811519F00E948605A7CF089527
:1020C000811531F09091AC06892B8093AC069ECFA0
:1020D0000895CF93C82F8115C1F08CEF8C0F813AF2
:1020E00080F580912001813021F48091F30687FDF5
:1020F0000EC0EAEEF1E08191C817F9F021E0E03F6F
:10210000F207C9F78C2F0DDB81DFCF910895EC2FFB
:10211000E695E695E695F0E0E051FE4F828190E08D
:102120004C2F477021E030E002C0220F331F4A9548
:10213000E2F782239323892B29F38C2F26DB66DF9A
:10214000E1CF80E28C0F883048F4C77081E001C095
:10215000880FCA95EAF70E948605D6CF8BE58C0FCB
:10216000833030F42C2F2452330BC9018ADACDCFBF
:10217000E8E5EC0FEB3148F4F0E0EE0FFF1FE1551E
:10218000FE4F80819181A5DAC0CF83E38C0F83312C
:1021900008F0BBCF61E08C2FC3DBB7CFCF93DF93C9
:1021A000EC01805E9109089720F060E670E12097CD
:1021B00011F46AE570E1CE010E948C048C2F89DF56
:1021C000DF91CF910895811541F19CEF980F913ADD
:1021D00010F4DBDA1BCF90E2980F983050F4877040
:1021E00091E001C0990F8A95EAF7892F0E948C052A
:1021F000F1CF9BE5980F933018F480E090E041CA4E
:1022000098E5980F9B3118F480E090E062CA93E360
:10221000980F933110F460E083CB08951F93CF9310
:10222000DF93182FEB0155DF209731F4812FCBDF9F
:10223000DF91CF911F9108958FE99FE00197F1F70A
:1022400000C000002197F0CF811519F00E948C0585
:10225000DDCE0895811539F080959091AC068923E3
:102260008093AC06D3CE089580918D05811521F021
:1022700082E2F0DF10928D0508951092A8068091F9
:102280002001813011F58091F30687FF1EC0E2EF37
:10229000F1E08EE1DF011D928A95E9F780E090E0A0
:1022A000F0D980E090E015DA1092AC06AFDE86E05F
:1022B000EDE7F5E0DF011D928A95E9F710927B05C5
:1022C00010927A0510927C0502CBEAEEF1E086E0EE
:1022D000E1CFD3DF2FEF84E39CE02150804090409A
:1022E000E1F700C0000088E19CE00FB6F894A895E3
:1022F000809360000FBE90936000FFCFAAE2B0E031
:10230000E4E8F1E10C94713288E192E0FC0101967D
:102310002091F100208322E080329207B9F780916A
:102320001902893009F457C0C8F4823009F4B2C0E8
:10233000833009F482C0813081F18091E80083FF0D
:10234000E6C080911802909119029A3008F0DFC01F
:10235000E92FF0E0EA5DFB4C0C9449328A3009F435
:1023600089C08B3051F780911802813231F780910A
:102370001C0290911D02892B01F78091E800877F54
:102380008093E8002EDC81E090911A02911101C047
:1023900080E08093200171DFD0CF80911802813AD4
:1023A00061F68091E800877F8093E80080911C02AD
:1023B00090911D02892B59F060E080E090E070E080
:1023C000B7DB8091E8008B778093E800B6CF68E0B8
:1023D00080E292E0F4CF80911802813209F0ADCF13
:1023E00080911C0290911D028D7F892B09F0A5CF51
:1023F0008091E800877F8093E8008091E80082FF69
:1024000017C09091F3008091F200029731F480910F
:10241000F100813011F0863021F48091F100809339
:102420001F018091E8008B778093E800DADB85CF8D
:10243000809122058111E1CF80CF80911802813AED
:1024400009F07BCF80911C0290911D02892B09F02D
:1024500074CF8091E800877F8093E8008091E80046
:1024600080FFFCCF809120018093F1008091E800F3
:102470008E77DACF80911802813209F05ECF809199
:10248000E800877F8093E800ACDB80911B0280939B
:102490001E0153CF80911802813A09F04ECF8091EE
:1024A000E800877F8093E8008091E80080FFFCCF00
:1024B00080911E01D9CF803889F0823841F5809112
:1024C0001C028F70873018F58093E9008091EB0033
:1024D00085FB882780F91092E90006C08091DB0413
:1024E000880F90911502892B9091E800977F909327
:1024F000E8008093F1001092F1008091E8008E775F
:1025000023C0811116C080911A02813009F1809197
:10251000E80083FF0AC08091E800877F8093E8008D
:102520008091EB0080628093EB00AA96E3E00C942C
:102530008D32823061F780911A02811581F01092FC
:10254000E9008091E800877F8093E8004ADBDFCFD5
:1025500081E0933009F080E08093DB04F0CF80913C
:102560001C028F702FEF280F263088F68093E90029
:102570002091EB0020FFE3CF933031F48091EB000A
:1025800080628093EB00DBCF9091EB0090619093A1
:10259000EB0021E030E0A90102C0440F551F8A95ED
:1025A000E2F74093EA001092EA008091EB00886025
:1025B000E8CF8111ACCF10911A021F778091E30010
:1025C0008078812B8093E3008091E800877F80935F
:1025D000E80007DB8091E80080FFFCCF8091E300FA
:1025E00080688093E30083E0111101C082E0809352
:1025F00022058DCF8058823008F089CF80911A0251
:1026000090911B028C3D53E0950791F583E08A83FE
:102610008AE289834FB7F894DE01139620E03EE00A
:1026200051E2E32FF0E050935700849120FF03C064
:1026300082958F703F5F8F708A30C0F0895C90E028
:102640008D939D932F5F243161F74FBF8091E800F8
:10265000877F8093E8006AE270E0CE01019668DA35
:102660008091E8008B778093E80051CF805DE7CFC1
:10267000292F33272330310509F44EC078F5213056
:10268000310509F488C08BE590E0E8E7F2E02230FC
:10269000310509F03CCF2091E800277F2093E80026
:1026A00020911E0230911F028217930708F49C01AB
:1026B00040E02115310509F073C0411171C08091CE
:1026C000E80082FDCDCF80912205811549F2853049
:1026D00039F28091E80083FFF2CFC2CF80911C02D3
:1026E00090911D022132310509F446C02232310594
:1026F00009F00DCF8330910508F009CFFC01EE0FF2
:10270000FF1FE25DFE4F0190F081E02D855D9E4F41
:10271000DC018C9190E010C09C013327823021F1C4
:102720002330310568F4232BB9F4EBE1F3E0E491B5
:102730008E2F90E0EBE1F3E0009709F4E8CEABCF09
:102740002330310509F0E3CEE5EEF2E0E4918E2F7F
:1027500090E0E5EEF2E0F0CFE3E1F3E0E4918E2FDC
:1027600090E0E3E1F3E0E8CFE3E0F3E0E4918E2FE3
:1027700090E0E3E0F3E0E0CF8330910508F0C7CECE
:10278000FC01EE0FFF1FEC5CFE4F0190F081E02D8D
:1027900089E090E080CF82E190E0E3EDF2E07BCF52
:1027A00080912205811509F45BCF853009F458CF5B
:1027B0008091E80083FD54CF8091E80082FD7FCFB7
:1027C0008091E80080FF75CF9091F3008091F20036
:1027D0002115310519F08830910550F041E0089736
:1027E00009F040E08091E8008E778093E80061CFA7
:1027F00044914093F1003196215031090196E8CF80
:10280000803809F084CE8091E800877F8093E800CB
:10281000809116028093F10070CE811178CE1091D4
:102820001A02123008F073CE8091E800877F8093FF
:10283000E80010931602D5D91115D9F084E08093E1
:10284000220542E061EC81E049DA42E261EC84E099
:1028500045DA42E261EC82E041DA42E260EC83E098
:102860003DDA80912205843051F482E08093210189
:102870004ECE8091E30087FDE1CF81E0E0CF81E0A3
:10288000F5CFCF93DF93EC014A855B856E857F851D
:102890000E942D0B9B8190958091AC06892380939B
:1028A000AC068C810E948C05B1DB86E0FE011192A2
:1028B0008A95E9F7DF91CF910895CF93DF93EC01EB
:1028C0008D8181FD13C082608D838091AC069B81D8
:1028D000892B8093AC068C810E94860597DB488506
:1028E00059856E857F85CE010E942D0B109297062B
:1028F000109296068D8180FD02C0CE01C2DFDF916D
:10290000CF9108951F93CF93DF93182FA0910C06BA
:10291000B0910D06109709F448C010920F0610925E
:102920000E0610929205109291051696CD91DC91AB
:102930001797CE019A9581159F4108F4D07ED1E07A
:10294000C11101C0D0E01996ED91FC911A97309712
:1029500031F01B966D917C9180E00995D823D115BB
:1029600039F08CEF8C0F813A20F58C2F0E94C50B2B
:102970001115A1F0E0910C06F0910D06808584FD03
:102980000DC080910B06811549F0808191819C01D9
:10299000215031092F333E4708F489D837DB109294
:1029A0000D0610920C0610920B06DF91CF911F912D
:1029B00008952CDB8C2F07DCDBCF0F931F93CF9375
:1029C000DF93833030F56B3020F5493010F5C42F9C
:1029D000D0E0CC0FDD1F22E1629FC00DD11D11247C
:1029E00036EC839FC00DD11D1124CE0189960E9423
:1029F0005E33082F10E0102F0027CE018A960E9428
:102A00005E339801282BC901DF91CF911F910F915F
:102A1000089580E090E0F8CF462F672F209125059C
:102A200030912605232B81F4703F39F4403F61F447
:102A3000809123059091240508957B3028F4493036
:102A400018F4833008F4B9CF80E090E00895A0E056
:102A5000B0E0EDE2F5E10C946D327C010091AB0643
:102A60008091AA06082BC2E0D0E010E0C8010C2E2D
:102A700002C0959587950A94E2F780FD09C02197D9
:102A8000A8F7D12C8D2DCDB7DEB7E7E00C948932B5
:102A9000DC2EB7018C2FC0DF0E949206019779F3DC
:102AA000F1CF0F931F93CF93FC018581008111819A
:102AB000811581F0611571F0C801C9DFC82F682F39
:102AC000C8010E94D804B8018C2FA6DFCF911F91B6
:102AD0000F910895C8010E940E05C82FF4CFCF931F
:102AE000DF93D82FC92FB3DF6D2F7C2F95DF0E9486
:102AF0009206DF91CF910895FC018481811599F0B0
:102B000080819181ECDF282F92959F70963099F00B
:102B100060F4925F9F70923030F4203FB1F038F44F
:102B200081E0283E38F080E008959A5FF3CF81E09D
:102B3000243FC9F7089591E0213F09F090E081E03A
:102B4000283E08F080E0892B089581E00895382F11
:102B5000292FCB01A32FB22F853E9105A105B105E9
:102B600020F4855E9C4F0C945E3380E0089585E2EE
:102B700090E00E945E338D3D89F486E290E00E94F1
:102B80005E33823F59F487E290E00E945E3391E029
:102B9000893609F090E0892F8170089580E0FCCF9C
:102BA000A0E0B0E0E6EDF5E10C946B32EC01888139
:102BB000811509F1813009F045C08981813051F4D6
:102BC0008A81239660E570E0893311F060E070E05F
:102BD00025DBEDCF823021F48A8123967ADAE7CFA4
:102BE000833021F48A812396EEDAE1CF843041F0FC
:102BF00022968111DCCFCDB7DEB7E9E00C948732A5
:102C00008A81239620E030E09AE0682F6053770BAA
:102C1000AB016A30710560F02115310551F3EFE920
:102C2000FFE03197F1F700C0000021503109F4CFE7
:102C3000929FB001939F700D11249A01260F371FA8
:102C40008991E3CFE82FF0E0E850FE4FB490282FB1
:102C500026952695269530E0F901E851FE4FE4903F
:102C60008770F12C082E02C0F594E7940A94E2F7DD
:102C7000E0FAEE24FF24E0F8F901E852FE4FC49098
:102C8000D12C082E02C0D594C7940A94E2F7C0FA5A
:102C9000CC24DD24C0F8F901E853FE4F049110E084
:102CA00002C0159507958A95E2F701701127E11486
:102CB000F10411F081EE0DDAC114D10411F086EEA9
:102CC00008DA60E070E08B2DA9DAC114D10411F0AC
:102CD00086EE79DAE114F10411F081EE74DA01156F
:102CE000110521F060E070E08CE298DA21965FCF68
:102CF000AAE0B0E0EEE7F6E10C946732C090200560
:102D0000D090210581E090E09093210580932005EB
:102D1000812C912C10E0540100E019C021E030E03A
:102D2000123021F0F701859195919C01472D602F7C
:102D3000812F45D9739422E0E20EF11C39E0731221
:102D4000EDCF0F5F89E0A80EB11C0B3049F0C50133
:102D5000880F991FFC01E15EFC4F7F01712CDECFD3
:102D60001F5FF3E68F0E911C1330A9F61A821982A9
:102D70001C821B821E821D8218861F8288EC90E0B6
:102D80009A8789870BE712E09E012F5F3F4F7901F9
:102D90004AE050E0B801C7010E949D33065F1F4F13
:102DA00057010B3C32E0130799F789E0F7011192C4
:102DB0008A95E9F78FEF9FEF9E838D8387E08A875F
:102DC0004AE050E0B801C5010E949D33065F1F4FE5
:102DD0000B31F3E01F07A1F7D0922105C092200527
:102DE0002A96EDE00C948332AAE0B0E0EAEFF6E137
:102DF0000C946A3203E915E08BECE82E82E0F82EA1
:102E000097E0B92E23E2C22E23E0D22EAA24A39467
:102E10004AE050E0B701CE0101960E944E33F8011E
:102E20003896DF018B2D1D928A95E9F789819A8169
:102E3000D80111969C938E938F8112968C93129742
:102E40008D8113968C931397888514968C93149781
:102E5000898515968C9315978B819C8117969C93E9
:102E60008E9316978A8587FD04C01E96DC92CE92BB
:102E70001D9780FF02C0F801A08681FF07C0D8011E
:102E800018969C911897926018969C9382FF04C0A4
:102E9000F80190859460908783FF07C0D801189649
:102EA0009C911897986018969C9384FF04C0F80131
:102EB00090859061908785FF07C0D80118968C9106
:102EC0001897806218968C93BAE0EB0EF11C015FA4
:102ED0001F4FEBE1EE16E3E0FE0609F099CF2A96CC
:102EE000EAE00C948632282FCB01283070F44AE0B7
:102EF000249F90011124B90165587D4F4AE050E0AC
:102F00000E944E3380E090E008958FEF9FEF089588
:102F1000AAE0B0E0EEE8F7E10C9472329C0197551C
:102F20008115914068F4BE016F5F7F4F822FDBDF18
:102F3000892B31F489859A852A96E2E00C948E32A9
:102F400088EC90E0F9CFA0E0B0E0E9EAF7E10C947A
:102F50006D32162FD72FC42FD22E8115A1F040939A
:102F60009A060E94F40B9093140280931302C77088
:102F700081E001C0880FCA95EAF79CD8CDB7DEB7CB
:102F8000E7E00C94893290919A06491335C0E0909D
:102F90001302F09014020E94F40B9C012E193F09B9
:102FA0007901812F9D2FB4DFE816F90628F5D0E2CC
:102FB000DD0DCD1591F0C77011E0812F01C0880F94
:102FC000CA95EAF741D9D83040F48D2D877001C0F9
:102FD000110F8A95EAF7812F6DD860E070E0802F9D
:102FE0001DD9D83058F62D2D277081E001C0880FEB
:102FF0002A95EAF729D9C2CFC77081E001C0880FAE
:10300000CA95EAF7F7CFA0E0B0E0E9E0F8E10C9468
:103010006632FC018280648081E08483EBEAF4E024
:103020009490EAE2F5E0E4910091A106069501583A
:1030300010E0000F111F012F1127CCE2D3E0C12CAB
:10304000D12CAA24AA94B12C77247A94E919EE2ED3
:10305000F12C83E0881630F480919F06888380915C
:10306000A006898361101AC01B821A824A81453BDF
:1030700008F044EB9601698188810E9431088FEF46
:10308000C81AD80A259681E5C816D10411F70E94FE
:103090005408CDB7DEB7EEE00C9482328B818115F7
:1030A000E9F081508B83789EC00111246C8170E01F
:1030B0000E942232FB01FF27E555FB4F8491E82F48
:1030C000E9197E9EC0011124B7010E94223280912D
:1030D000A106689FB00111247A83C8CF0E941633DD
:1030E000B5010E943632801791070CF0BFCF83E004
:1030F000881688F00E941633B5010E943632888304
:103100000E9416332091A0062695622F70E00E943F
:103110003632280F29831A828091A106893C20F03B
:1031200088EC8C838B83A2CF8431D8F784E1F9CFEC
:103130000F93CF93DF93CEE9D6E0488159816A811E
:103140007B8188E090E00E949133288139814A8117
:103150005B816C817D818E819F8100E20E94B4320F
:10316000622F83E290E00E947F33DF91CF910F9135
:103170000895EEE9F6E085E0808311828FEF828387
:1031800084EB83831482CF01D3CF8091A206833056
:1031900018F48F5F8093A2068EE996E0C9CF8091E4
:1031A000A206811519F081508093A2068EE996E05F
:1031B000BFCFA0E0B0E0EFEDF8E10C946732082F4C
:1031C000F62E142FE22E90919E0690FF26C0E92F36
:1031D000E695E695AE2FB0E0A65CBE4F8C9180934D
:1031E0009C069C7F9430F1F4842F453B08F084EBDF
:1031F000602F7F2D0E94AA07962F672F482F892FB7
:103200000E94690800939F06F092A0061093A10601
:10321000E11419F08EE996E08BDFCDB7DEB7EDE073
:103220000C948332823019F41091A106EBCF8630D2
:1032300019F400919F06E6CF8930D9F3893111F74F
:10324000E9518E2F8170782EE695F0E0E555FA4F22
:10325000E491CE2FD0E0A12CB12CC12CD12C81E552
:10326000882E912CC501B4010E942232802F71104A
:1032700015C0860F412F153B08F044EB96016F2DCA
:103280000E9431088FEFC81AD80AAC0EBD1E81E526
:10329000C816D10439F70E945408B4CF861BEACF70
:1032A000EEE9F6E0818121E043816281885F81CF90
:1032B000EEE9F6E0818121E043816281885079CF97
:1032C000EEE9F6E0628128E0620F08F46FEF21E09A
:1032D000438181816ECFEEE9F6E0628128E0621BD6
:1032E00008F460E021E04381818163CFEEE9F6E0FC
:1032F000438128E0420F08F44FEF21E06281818191
:1033000058CFEEE9F6E0438128E0421B08F440E0A4
:1033100021E0628181814DCF90919E0690FF2CC06B
:10332000811559F18B3258F58F73880F880F909162
:103330009E069370892B80939E06611519F08EE985
:1033400096E0F6DE60919E066695669570E04BE02D
:1033500050E087E091E00E942D33892B91F010928C
:103360009D0681E08093FE0420E04091A1066091DB
:10337000A00680919F061DCF089581E0D6CF8AE2F6
:10338000D4CF81E080939D060E94F40B9093FC04BF
:103390008093FB04E6CF80919E06869586958F5F8D
:1033A0008B3208F081E061E0B7CF80919E06869570
:1033B00086958A9509F48AE261E0AECFACE0B0E090
:1033C000E4EEF9E10C9463327C01DC0114968C91FB
:1033D000811509F4BFC161E0C70163DB8C01F7010E
:1033E0008581811521F1809196069091970600972D
:1033F000F1F008171907D9F0FC01FF27887F9927FA
:10340000892B09F072C0A4E0EE0FFF1FAA95E1F727
:10341000EA5EF94F85818460858311830083CF0143
:103420004CDA1092AC0661E0C7013BDB8C01D7019E
:1034300015968C91811509F4E3C0C801975780381F
:10344000910508F06CC1003108F073C164EE70E0C2
:1034500080E090E07CDB81116CC1812C912C5401C7
:10346000011146C004E09E012F5F3F4F6901D60164
:10347000E02F1D92EA95E9F724013501FFEF4F1A7D
:103480005F0A6F0A7F0AC501B40161DB8983811578
:1034900009F44FC1813009F0B0C0A50194012E5F3D
:1034A0003F4F4F4F5F4F2D833E834F835887C3015C
:1034B000B2014DDB182F8A83811509F43AC18FEFD1
:1034C000810F833078F56D817E818F8198853FDB18
:1034D0008B83811511F0C60163DB2401350133E0D4
:1034E000430E511C611C711C1AC0E0E0F0E092CF49
:1034F000B5EE8B169104A104B10409F41AC1C501FB
:10350000B40125DBEFEF8E1A9E0AAE0ABE0A8111C6
:10351000EFCF0150A5CF4D805E806F80788453013E
:103520004201A5CF8BEF810F833090F52401350147
:1035300043E0440E511C611C711C6D817E818F81A2
:10354000988505DB8B83811551F3C301B201FFDA46
:103550008C83811108C02401350154E0450E511CB3
:10356000611C711CDCCF8B819C818130AFEF9A078D
:1035700010F0982F8827163029F0173031F00E946C
:103580007526E9CF0E942226E6CF0E944326E3CF8C
:10359000143009F0C0CF6D817E818F819885D7DA94
:1035A000182F24013501B4E04B0E511C611C711C15
:1035B000C501B4016D5F7F4F8F4F9F4FC8DA111562
:1035C00009F4B7C0811509F4B4C08150990B4FEFCD
:1035D000489F9001499F300D1124E12FE150FF0BCE
:1035E0002E0F3F1F2150310908F499CF8FE99FE03A
:1035F0000197F1F700C00000F5CFC601D1DA8FCFF7
:103600000115A7E51A0708F4B9C00115B8E51B07AD
:1036100010F00C9455236801E7E5DE1A63E875E0C5
:103620008C2D61DC892B31F5C601E4E0880F991FF0
:10363000EA95E1F7FC01EA5EF94F2281213009F0B9
:103640005AC02091830530918405232B99F0209155
:10365000850530918605232B69F0209187053091EF
:1036600088054091890550918A05242B352B232B01
:1036700009F44BC080918D05811509F404C1C090F7
:10368000A806D090A7060E94F40B88579C4E9093F2
:103690008F0580938E05F7018581811509F4F3C0AC
:1036A0008D2D8C298D79811120C10115F0E51F0721
:1036B00008F0BBC0011520E4120708F01DC1063E4A
:1036C000110509F4E0C0C80190528115904208F03C
:1036D0001AC1D70116968C91803108F4FEC0C8013A
:1036E00099271092AC068D32910509F0B7C082E09F
:1036F0008093AC060CC1223009F0BCCF2091870525
:1037000030918805232B09F4B5CFFC01E55EF94F14
:1037100020812E7F20838A5E994FCFD8ABCF03378D
:10372000FCE71F0759F580918D058115B9F00E94BE
:1037300034118091AD068770811561F0D70115961F
:103740008C91811539F08091F40682FF03C082E0EC
:103750000E946B052C96E1E10C947F321092A80632
:103760000E9494050E94F40B88579C4E90938F05FD
:1037700080938E0581E080938D05DBCF023A22E5B0
:103780001207C1F158F4C80190528115904218F106
:10379000013E110579F1053E110503C0023B52E5DA
:1037A000150709F067CF25EE30E02770332781E059
:1037B00090E001C0880F2A95EAF72091900530919A
:1037C0008D053115F9F0F70135813115B1F0282B50
:1037D00020939005AECFD70116968C91803108F0DA
:1037E00049CF812F99278F7199278230910511F048
:1037F0004297D7CF21EE30E0D8CF809582238093B7
:10380000900597CF322F3823311509F433CF982FF5
:1038100090959223909390050E948C05D701159660
:103820008C91811509F485CF25CF003EB2E51B07A9
:1038300008F046C0003CE2E51E0728F5003AF2E534
:103840001F07E8F4003622E51207E8F4C801925594
:1038500080349105C0F01092AC06C8018E329105FB
:1038600008F062C08832910508F04FC08E31910592
:1038700008F04DC004974A9708F439CF36C0043B8E
:1038800032E5130741F7F7013580311409F456C0CA
:103890000E35FCE71F0709F44DC00F352CE7120762
:1038A00051F00D353CE7130709F048C08091220123
:1038B000811509F43FC01092220180E023D839CF4E
:1038C00009374CE7140728F407375CE71507D8F6E3
:1038D000C2CF0B378CE71807D5CF812F8F7184317A
:1038E00091F2863111F41092AC060E94341180914D
:1038F00090050E948605C7CFD70116968C9180311E
:1039000008F0EDCEC0CFC801ECCE8A9771F7809158
:103910009005811531F08091AC0692E08927809363
:10392000AC060E940610AFCF8C34910581F38D3226
:103930009240ECCF81E080932201FBCE8091220166
:10394000811169C0C80197558115914008F0FFC0E9
:103950005801F8EFAF22BB24A114B10409F0E9CE5D
:10396000F801FF2754E0EE0FFF1F5A95E1F79F0182
:103970002A5E394F6901D70115968C91E55EF94FA2
:10398000908180FB90F99083811509F4D9C10E9440
:10399000F40B9093990680939806F60182818F5FCD
:1039A00082838091AC069091A806892B83838091B5
:1039B000A70684834681578166857785C6010E9464
:1039C0002D0BD60115968C9181FF5801B092970668
:1039D000A0929606D70115969C91911509F47EC682
:1039E00010929A06980130572332310508F061C6CB
:1039F00084E090E00E946B339093F4068093F3068A
:103A0000F801E150F047E232F10508F0E1C1E05D74
:103A1000FB4C0C944932380150EE651A71085090F5
:103A2000A9068091A806582A8091A706582A88E0FE
:103A30006816710408F05EC098012770332781E092
:103A400090E001C0880F2A95EAF7311409F44FC0BD
:103A5000582AD7018D919C910E940E0521E030E0FB
:103A6000F90102C0EE0FFF1F8A95E2F7FC87EB8792
:103A700020910C0630910D063E832D834091140653
:103A8000509115065A87498763E9C62E65E0D62E00
:103A9000A12CB12C511005C0D60112968C91811128
:103AA0001BC0F601838190E02B853C858223932304
:103AB000892B91F08085982F9770911101C087E034
:103AC00038E06316710408F066C0311409F45FC071
:103AD00086958170811164C09FEFA91AB90AAFE081
:103AE000CA0ED11CB8E0AB16B104A1F61CC080957B
:103AF0005822AFCF311038C080911406909115062E
:103B00000817190781F410921506109214061092E6
:103B100010061092110610921206109213061092BF
:103B20000F0610920E0680910C0690910D060097DC
:103B300009F408CFE8E06E16710408F0EBC0652DBB
:103B40000E94920A811103C081E00E948214F70151
:103B50008581F801E851FC47E730F10508F03ACFDC
:103B6000EE5AFB4C0C944932109315060093140640
:103B70000E944B0D609310067093110680931206FD
:103B80009093130610920F0610920E0662CF82FBDE
:103B9000882780F99FCF311409F49ECF80FF9CCFF6
:103BA000D6018D909C900815190519F4311409F46B
:103BB00093CFED81FE81EC15FD0509F48DCFD60183
:103BC0001D96ED91FC91309721F08081811509F4CB
:103BD00083CF652DC6010E94920A811509F47CCF1E
:103BE00081E00815190509F080E0482E4320811472
:103BF000910441F0411006C0E985FA858E169F06B2
:103C000009F06ACF80E00E948214D0920D06C09223
:103C10000C0681E080930B068FE08A9DF0018B9D5E
:103C2000F00D1124ED56FA4F8581809392054110D5
:103C30000EC08114910459F0808191819C0124501F
:103C40003109213A310508F049C00E94C50B8FE0C7
:103C50008A9DF0018B9DF00D1124ED56FA4FC68020
:103C6000D780C6019A9581159F4110F420EED2228B
:103C700099249394C60101978F339E4708F0912CA5
:103C80008FE08A9DD0018B9DB00D1124AD56BA4FA7
:103C90001996ED91FC911A97309731F01B966D9122
:103CA0007C9181E0099598229114A9F08FE08A9D7A
:103CB000F0018B9DF00D1124ED56FA4F868197810E
:103CC0000E94620480939105C60148E06416710465
:103CD00040F40E94570D0E9406100AC00E94E31093
:103CE000B6CF0497813A910548F48C2D0E94910B30
:103CF000411409F427CE0E9406101BCD0E94061025
:103D00008FE39CE90197F1F700C000008C2D0E9421
:103D10006910EECFDC012D913C910217130741F49D
:103D2000311009C010920B0680E00E9482140ACE66
:103D3000311409F407CEFC01808585FD03CEF4CF54
:103D4000F9014485558566857785C9010E942D0B4B
:103D5000D60115968C9181FF3DCEC6010E9441147B
:103D600080919606909197060817190709F032CEB0
:103D700010929706109296062DCE06E221EE41EEA5
:103D80006AE17CE7E0D8D5CC07E225EE45EE6BE1B1
:103D90007CE7F8CF06E221EE40EE68E17CE7F2CF67
:103DA00007E225EE44EE69E17CE7ECCF06E221EE86
:103DB00042EE6CE17CE7E6CF07E225EE46EE6DE1F0
:103DC0007CE7E0CF08E221E045EE6EE17CE7DACF68
:103DD0008091F30681608093F3066091F306709101
:103DE000F40684E090E00E9499330E943D11A1CC3A
:103DF0008091F40688608093F406EFCF8091F306FB
:103E00008260E9CF8091F3068460E5CF8091F3066C
:103E10008860E1CF8091F4068160EDCF8091F40657
:103E20008260E9CF8091F3068061D5CF8091F3065F
:103E30008062D1CF8091F3068064CDCF0E943D1186
:103E40008091F3068068C7CF8091F3068C60C3CF62
:103E50008091F4068360CFCF8091F3068E7FBBCF35
:103E60008091F406877FC7CF8091F3068D7FB3CF13
:103E70008091F3068B7FAFCF8091F306877FABCF26
:103E80008091F4068E7FB7CF8091F4068D7FB3CFFB
:103E90008091F3068F7E9FCF8091F3068F7D9BCF1D
:103EA0008091F3068F7B97CF0E943D118091F3069E
:103EB0008F7791CF8091F306837F8DCF8091F40629
:103EC0008C7F99CF8091F306992782FF939590FB81
:103ED00082F990FB83F97FCF8091F406982F90951B
:103EE00090FB80F990FB81F986CF9091F306892FA2
:103EF0008F7B96FF80646FCF0E943D119091F306F7
:103F0000892F97FB87F9805866CF61E08EE090E0BB
:103F10000E947F3362CF60E0F9CF9091F306892F42
:103F20008F7E94FF806157CF9091F306892F8E7F0B
:103F300090FF816050CF9091F406892F877F93FF87
:103F4000886059CF89E2C7C389E2D3C38272F8017E
:103F5000E052F847EB30F10508F04CC0E75AFB4C53
:103F60000C9449320737BCE71B0709F047C081E0D2
:103F70000E94CA0465C080919E0680FF0BC08E7FA0
:103F800080939E068EE996E0D3D810929D060E94FB
:103F90005408CFCB816080939E0661E0869586951C
:103FA000BBD9C7CB811521F000DAC3CB8115E1F372
:103FB000F2D9BFCB811521F07BD9BBCB8115E1F3C1
:103FC0006FD9B7CB811521F086D9B3CB8115E1F339
:103FD00077D9AFCB811521F094D9ABCB8115E1F323
:103FE00085D9A7CB811521F0DAD8A3CB8115E1F3D0
:103FF000CCD89FCB0737ECE71E07F9F00837FCE772
:104000001F0721F19801205E32452032310518F555
:10401000911121C00F7181E090E09C0102C0220F3C
:10402000331F0A95E2F78901622F83E090E00E9436
:104030007F33802F0E94BA047CCB81E00E94C004B1
:1040400043E062E081E00E94420573CB82E091157B
:1040500009F48ECFF3CF4091A6068091AB06282FAE
:1040600030E02095309570E024233723232B19F07E
:1040700048234093A6060B373CE7130741F49115FC
:1040800009F457CB0E9495040E94B30A52CB003426
:1040900042E5140708F055C0003252E5150708F054
:1040A00057C0011580E5180750F50115A0E41A075F
:1040B00008F064C0911509F479C00A35FCE71F07C0
:1040C00009F4DDC008F0C2C001303CE7130709F471
:1040D000D4C003304CE7140709F4C9C001151C47CC
:1040E00009F064C00E943D11AFEFB4E3ECE0A150D1
:1040F000B040E040E1F700C000000E943D0F980191
:10410000305521153240B0F6980145E03695279597
:104110004A95E1F7822F8F702091A60630E041E0AA
:1041200050E0082E02C0440F551F0A94E2F72423E2
:104130003523232B09F4BECF9111A6CF1092A806E8
:10414000DACD9801205C32452032310508F0B2CF3B
:10415000802F8F712091A60630E041E050E0082EBC
:1041600002C0440F551F0A94E2F724233523232B62
:1041700009F4A0CF911509F4DCCA86CFF701868136
:10418000803108F097CF911111C0212F2F7081E05D
:1041900090E002C0880F991F2A95E2F72091A606A9
:1041A00030E082239323892B09F0C3CAF70185816C
:1041B000C080D180811509F466C0C6010E94271510
:1041C000182F682FC6010E94D804B601812F0E94C3
:1041D0000C150E9492068C01D7011596BC9015977C
:1041E0001696AC90A2942FE0A2228091AD06877023
:1041F000811501F1CB2CB114F1F0812F807F803437
:1042000061F080E2800F8830A8F0812F807E8032BC
:1042100021F4023078F0A11469F08091F40682FF55
:1042200009C082E00E946B058091AD068770CC24A6
:10423000C3948111C12CE12FE295EF70103C08F07E
:1042400082C0F0E0EC59FB4C0C9449320B358CE702
:104250001807B9F08091F406002482FF0394802DA2
:104260000C351C4709F0A2CF0E94C80F9FCF6FEFFB
:104270007FEF80E090E00E9499330E94691181E015
:10428000F3CF80E0F1CFC6010E940E05182F9DCF1D
:10429000B12FBF70DB2E103118F0D29490EFD922DD
:1042A000B114A9F0D11459F080E2800F883010F0D9
:1042B000011107C08D2D0E9486050E940610802FD7
:1042C00040C08091AC068D298093AC06F6CF802F3C
:1042D0000E94E310D114B9F180E2800F883010F011
:1042E000011104C08D2D0E948C0506C0D0948091D0
:1042F000AC068D218093AC060E94061024C0E12FED
:10430000EF70DE2E107F103219F0D29480EFD82299
:10431000011549F0013009F482C0B11409F48EC0CE
:10432000A114A1F1CCCF8091F40682FD2BC0B11471
:1043300019F1D11429F08D2D0E9486050E940610D6
:1043400080E00E946910C11409F4DAC08091AD06C2
:1043500080FDD6C0D70115961C92869586958695C8
:104360000E94C004C7012AD88091AD068695869523
:1043700086950E94CA04C4C080E00E94E310D11454
:1043800011F3B0CFB11469F1A11004C08D2D0E94BA
:104390005A10D9CFF1E0AF1210C01091A7068D2DA1
:1043A0008123D81681F20E94F40B9093B10680937A
:1043B000B0061D291093A706C6CF25E0A212C3CFD1
:1043C0008D2D0E945A108D2D0E94520C8091A906AD
:1043D0009D2D9823D91609F4B6CF8D298093A9066F
:1043E000B2CFA11012C08D2D0E9424118D2D0E94DC
:1043F000520C8091A9069D2D9823911509F4A3CF05
:10440000D094D822D092A9069ECF31E0A3129BCFA0
:104410008091A8068D21811509F495CFE4CFB114C0
:1044200029F046E0A41608F08ECFB0CF55E0A516CF
:1044300008F089CF8D2D0E94241185CFA114D1F3CE
:10444000093349F48FEF97EEA3E081509040A040EC
:10445000E1F700C00000802F0E94E31074CF812F8D
:10446000869586958370811561F0813009F06BCF58
:10447000C8019370B11002C080E090E00E94690B07
:1044800062CFC8019370B11002C080E090E00E943A
:10449000410B59CF6B2D802F0E94900C54CF812F50
:1044A000837081113AC0B11027C0402F42954695C4
:1044B0004770440F440F802F8F70042E01C0880F67
:1044C0000A94EAF7202F207104FF07C02FE030E0A4
:1044D00001C0220F4A95EAF720951695169513709C
:1044E0001230B1F0133091F03091AA06113069F01A
:1044F000822B83230E94BA040E94320B0E94A804DC
:1045000060E0C7010E94511525C9832B822BF2CF91
:10451000822B9091AA068927EDCFB11451F110FF9B
:10452000EBCF402F429546954770440F440F802FA4
:104530008F70042E01C0880F0A94EAF7202F207193
:1045400004FF07C02FE030E001C0220F4A95EAF7D0
:104550002095169516951370123089F0133069F076
:104560003091AB06113041F0822B83230E94BD04B1
:10457000C3CF8230B0F6C0CF832B822BF7CF822BF4
:104580009091AB068927F2CF1F70B11439F0812FBB
:104590000E94C004802F0E945A10AECF802F0E942C
:1045A0002411812F0E94CA04A7CF023F71F170F439
:1045B000003FC9F0013F91F0B11409F465C0A114A6
:1045C00009F45FC0802F0E94691096CF033F21F14C
:1045D000043F91F78091F40682FD2AC0812F8F71EC
:1045E000B11401F316C0B11469F0B5E0AB1608F0D0
:1045F00083CF1F7181E090E0012E01C0880F0A94E3
:10460000EAF7BECFE6E0AE16F2CF812F8F71B11080
:10461000C9CF0E94C00470CF80E0B11409F4A6CFC6
:104620001F7181E0012E01C0880F0A94EAF79ECF26
:10463000B114C1F08091AD068770843049F41092B6
:10464000AD061092AF061092AE06812F8F71AACFE1
:10465000F5E063E0AF1608F04FCF812F8F710E9415
:104660003E0C4ACF25E0A21640F01092AD06109203
:10467000AF061092AE0664E0F0CF81E00E946B05B9
:104680003BCF812F8F71C5CFA114F9F2093349F4C3
:104690003FEF47EE53E0315040405040E1F700C05B
:1046A0000000802F0E94E31027CF0337BCE71B07D1
:1046B000B9C88091A8060631ECE71E0709F046CC80
:1046C0008A7A91E0811101C090E090939B06811558
:1046D00009F438CC85E30E94910B0DCB0631FCE741
:1046E0001F0709F03FCC80919B06811509F42CCC63
:1046F00085E30E94C50BFFCAA0E0B0E0E2E8F3E268
:104700000C946D328091F206803108F049C080919E
:10471000F106811509F444C0C091B30687E0D82E94
:104720008091B2068C17E1F1EC2EF12CDC9EE001B9
:104730001124FE01EC54F94F84818115B1F191816E
:104740008091ED06981331C090818091EC0698130A
:104750002CC08581811129C0028113818091EE06D0
:104760009091EF06081B190B60E08CEE96E00E941A
:1047700051150E94881708171907B8F48091F2069E
:104780008F7080618093F206C654D94F88818F70F4
:10479000806188838CEE96E00E94DE190E9461059C
:1047A000CDB7DEB7E7E00C948932E7012196C770F8
:1047B000B7CFADE0B0E0EFEDF3E20C9465328C01E1
:1047C00086E0F801DE01189601900D928A95E1F7D6
:1047D000F801F580E4808CEE882E86E0982E80919A
:1047E000F006811117C0E11491F0F11409F455C1DC
:1047F000C8010E947C15811509F44FC187E0F801BA
:10480000ACEEB6E001900D928A95E1F775DFFF24DA
:10481000F39461C0A280B380D090F1068091EE063F
:104820009091EF063501681A790AD11409F4F0C0A5
:10483000C080518060E08CEE96E00E9451150E948D
:1048400088176816790608F09EC0E11401F380917C
:10485000ED06F8019181E090F206F0E1EF1608F024
:104860005BC0981317C09091EC06F80180819813F3
:1048700011C0F1104BC08E2D8F7080618093F206B5
:104880008CEE96E00E94DE198091F206F801868394
:10489000F12C21C0F1103AC040E0652D8C2D0E9412
:1048A000F80E40E0652D8C2D0E94F80EF82E811137
:1048B000EFCF888599850E946F15292F22952F703B
:1048C000903470F49F702230A0F09115B1F0F8018F
:1048D0009681903190F48F2D2D96EFE00C948132DB
:1048E0002A5F2F70223068F0C8010E94DE19FD2C6B
:1048F000F2CF911511F0811571F3805E883058F375
:10490000F3CF803F40F3815F8330F9CF8091F2068F
:1049100081608093F206BCCF981315C09091EC068D
:10492000F801808198130FC0F1100DC0E682C80114
:104930000E94DE1987E0F801ACEEB6E001900D921E
:104940008A95E1F764CFC8010E947C15811509F4AE
:10495000A4C0F11409F4A1C08091F206803208F4D9
:104960004DCF8091EC069091ED069A838983BC82AD
:10497000AB828091F0068D831E82EF82CE0101967C
:104980000E94DE193BCFD090F206F0E1DF1650F422
:104990008CEE96E00E94DE1987E0F40111928A9570
:1049A000E9F776CFE11409F432CF9091ED06F801E2
:1049B0008181981311C09091EC06808198130CC0EE
:1049C000F1100AC0D682C8010E94DE1987E0F40106
:1049D00011928A95E9F71BCFC8010E947C158115B9
:1049E00009F45BC0F11409F458C08091F2068032DA
:1049F00008F404CF8091EC069091ED069A838983A8
:104A0000BC82AB828091F0068D831E82DF82B6CF9E
:104A100060E08CEE96E00E9451150E94881768169F
:104A2000790608F0B9CFE11409F4F1CEF114A9F137
:104A30009091ED06F8018181981325C09091EC06C4
:104A40008081981320C08091EE069091EF06A81AFD
:104A5000B90AF8ECAF16B10408F06CCF8091F206F9
:104A600080FD68CF803108F465CFF8018683982FE8
:104A7000907F903F09F45BCF982F907F905F8F706D
:104A8000892B868354CFC8010E947C158111B6CE34
:104A90008091F20681608093F206C8010E94DE19BF
:104AA000B6CEABE1B0E0E7E5F5E20C9470324E8BA8
:104AB0005F8B688F798F8A8F192F9B8F911110923E
:104AC000AC061D8A86E0FE017696DE011F960190F7
:104AD0000D928A95E1F70A8D8091F40682FF1FC03E
:104AE0000E94F40B2091AE063091AF06821B930B0F
:104AF0008838934138F08091AD0682FD03C082E092
:104B00000E946B050E94F40B2091B0063091B10613
:104B1000821B930B8838934110F00E949405011575
:104B200061F00B8B1C8B61E0CE010F960E9451153A
:104B300061E0CE010F960E9451150B8B1C8B87E014
:104B4000FE013F96DE01189601900D928A95E1F7DD
:104B5000CE0108962EDE811110C02091B206309150
:104B6000B30687E0FE013896DE01119601900D92A2
:104B70008A95E1F78C8581110BC017E08091B3060F
:104B80009091B20689132BC06B96E4E00C948C32A2
:104B9000822F90E00196877099273817190671F4D3
:104BA0000E943D111092B2061092B30687E0ECEE1F
:104BB000F6E0DF011D928A95E9F7DFCF97E0929F3B
:104BC000D0011124AC54B94FFE01319601900D92E1
:104BD0009A95E1F78093B2060E946105CECF189FA7
:104BE000C00111248C54994FE4DD811569F2809144
:104BF000B30690E00196877099278093B306BECFE5
:104C0000A6E0B0E0E6E0F6E20C9470320E94F40B0D
:104C10008C0180912705909128058017910771F0EC
:104C200019821A820E94F40BBC0149815A8180E0EA
:104C300090E037DF10932805009327052696E4E0DF
:104C40000C948C32A6E0B0E0E8E2F6E20C9472320A
:104C50009093240580932305811520E2920730F478
:104C60000E94CE102696E2E00C948E3280EF89836B
:104C70008A830E94F40B8160BC0149815A8181E0E2
:104C800091E00FDFEFCFA6E0B0E0E9E4F6E20C94AC
:104C900070328C019093240580932305011580E2E6
:104CA0001807B0F4802F0E94E310C801805E9109BC
:104CB000089728F06AE271E10115110511F464E228
:104CC00071E1C8010E948C042696E4E00C948C32B9
:104CD00080EF89838A830E94F40B8160BC01498143
:104CE0005A8181E090E0DDDEEFCFCF93DF93D82FC4
:104CF000C92FA8DF8D2F9C2FC6DFDF91CF9108959C
:104D00000F931F93CF93DF938C01862F63E875E099
:104D10000E947317892B91F4C0918305D09184056B
:104D2000209761F0F8018281833039F4CE01DDDF14
:104D3000CE01DBDFCE01D9DF01C0E0F7DF91CF91FB
:104D40001F910F9108950F931F93CF93DF938C01C1
:104D5000EB0163E875E08C2F0E947317892B09F033
:104D600057C0FE01FF27D80112968C911297EC5D77
:104D7000FC4F8130A9F415968C9182FD4EC080FFC6
:104D80004CC082E0808380918505909186050097D4
:104D9000B9F480918305909184050097C9F110C002
:104DA0008230A1F515968C9182FD26C080FD0AC047
:104DB00083E0808380918705909188050097F1F0CA
:104DC00041DF26C084E080838091890590918A0527
:104DD0000097B1F78091830590918405009701F1C8
:104DE00084DF8091850590918605009749F7809131
:104DF000830590918405E4CF85E0808380918305CD
:104E000090918405009721F070DFF1CF86E08083D8
:104E1000DF91CF911F910F91089581E08083B9CFE9
:104E20008091850590918605B8CF0F931F93CF93FE
:104E3000DF938C01EB0163E875E08C2F0E94731700
:104E4000892B71F4DD27CC5DDC4F8881F80112825B
:104E500018828330E9F048F4813059F0823081F0D3
:104E6000DF91CF911F910F9108958430B1F085307B
:104E7000B9F78091830590918405009789F306C066
:104E80008091850590918605009799F3FCDEE8CF27
:104E90008091870590918805F7CF80918905909141
:104EA0008A05009799F720918305309184058091B8
:104EB00085059091860521153105F9F2009731F7A6
:104EC000C901E4CFA0E1B0E0E8E6F7E20C94643277
:104ED000FE01319680E1DF011D928A95E9F70FE02E
:104EE00010E09BE1A92E93E0B92E25EE422E512C25
:104EF000612C712C4F0173016201B1E14B16510419
:104F0000610471041CF080E1C82ED12CA601B5010A
:104F1000C4010E947033AC0CBD1C0D2C000CEE08BB
:104F2000FF084C185D086E087F080150104019F703
:104F30006096E0E10C9480326FEF85E290E00E9491
:104F40007F336FEF86E290E00E947F336FEF87E25E
:104F500090E00E947F3360E088E290E00E947F331F
:104F60000E947816AFDF6DED85E290E00E947F33FE
:104F700062EF86E290E00E947F3369E687E290E08C
:104F80000C947F338F929F92AF92BF92CF92DF9219
:104F9000EF92FF920F93CF93DF9388E090E00E940F
:104FA00066334B015C01CEE9D6E068839982AA8220
:104FB000BB821C821D821E821F8283E290E00E94BF
:104FC0005E33282F30E040E050E060E070E080E0A9
:104FD00090E000E20E949932282939294A295B2968
:104FE000288339834A835B836C837D838E839F838D
:104FF000DF91CF910F91FF90EF90DF90CF90BF9016
:10500000AF909F908F900895A6E1B0E0EAE0F8E2BB
:105010000C946632FE01319686E1DF011D928A957D
:10502000E9F705E611E09EE6C92E91E0D92EEE24BF
:10503000E394F12C9E2E8F2EAA24A394B12CF80178
:1050400081918F018F3F09F44BC0F894E82FE295CE
:10505000EF70F0E021A18F70A50102C0440F551F31
:105060008A95E2F7CA01922F982B91A392A180957D
:10507000892382A3789400C0AEE6B1E0692C782C35
:105080009701209530956D91F301819191913F01A8
:105090006F3F09F44BC0462F42954F70405E50E081
:1050A000FA01408150E06F7002C0559547956A95AE
:1050B000E2F740FD3BC08E299F29A30142505109D0
:1050C000FA0191838083F1E0A937BF07E1F6F80187
:1050D00082918F3F11F00E94900740EA4A95F1F7C4
:1050E000EE0CFF1CC016D10609F0A9CF46E150E036
:1050F000692D782D83EC94E00E943A33892BC9F016
:1051000086E1E92DF82DA3ECB4E001900D928A958B
:10511000E1F781E0809312020E94F40B9093110258
:10512000809310026696EEE00C94823282239323E1
:10513000C4CF809112028115A9F300911002109141
:1051400011020E94F40B801B910B059758F346E166
:1051500050E063EC74E08AE095E00E943A33892BDA
:1051600049F086E1E3ECF4E0AAE0B5E001900D92AD
:105170008A95E1F710921202D5CFCDB7DEB7AC9782
:105180000FB6F894DEBF0FBECDBF85B7806885BF70
:1051900085B7806885BF84B7877F84BF0FB6F894D2
:1051A000A8958091600088618093600010926000F3
:1051B0000FBE80E890E00FB6F89480936100909362
:1051C00061000FBE81E0809321018EE897E090930B
:1051D000E7018093E6010E946D0A0E94F4160E9486
:1051E000410E0E949E0E8091E20084608093E20056
:1051F000789480912205811599F08091E9001091B1
:10520000EC008F70179511271795182B1092E90055
:105210008091E80083FD0E947E111F701093E900C9
:1052200082E084BD93E095BD9AEF97BD80936E00B8
:105230000E94B715811101C07FDE05E611E0D8019B
:105240008D918D018F3F11F00E949007B1E00E36D5
:105250001B07A9F70EE611E089E7E82E81E0F82E9A
:10526000F80181918F018F3F11F00E949007E016A5
:10527000F106B1F786E1EAE0F5E0DF01282F1D92A3
:105280002A95E9F7E3ECF4E0DF011D928A95E9F74E
:1052900080E090E00E946B33833E9E4F21F40E9499
:1052A000B71581112AC063EE7EEF80E090E00E9486
:1052B000993360E082E090E00E947F3381E0809348
:1052C000AA0661E083E090E00E947F3360E074E131
:1052D00084E090E00E9499330E94B9182DDE40E0EE
:1052E00050E0BA018FE090E00E94913340E050E03E
:1052F000BA0183E190E00E94913382E090E00E9445
:105300005E338093DC0484E090E00E946B339093E2
:10531000F4068093F30678DEEFEFF6E721E0E15044
:10532000F0402040E1F700C000006EDE80910A05E9
:1053300080FF08C06FEF7FEF80E090E00E9499331C
:105340000E943D0F83E090E00E945E330E94BA0409
:10535000259A2D9A3E9A469A3F9A479A8091D90467
:1053600081111EC08EE996E00DDE80919E0684308C
:1053700028F40E94B9188EE996E004DE0E943F08E6
:1053800010929D060E94850A80919E0680FF05C0AE
:1053900060E0869586950E948C1981E08093D904FF
:1053A00082E191E090934A0580934905809122051E
:1053B00010E4853009F48DC027DEBDEDAB2EB4E0DE
:1053C000BB2E1AE0412E15E0512ED201F50121919C
:1053D00031918D919D9144E0E33FF40709F485C03C
:1053E00028173907A1F3AAE08A2EA5E09A2E10E02B
:1053F000D401ED90FD904D01F501619071905F0138
:105400006E147F0449F16E247F2400E0CC24C39401
:10541000D12CC60186219721892BB1F009831A83EB
:105420000E94F40B9C838B83F1E0FD8391E0960155
:105430002E213F21232B09F490E09E8349815A813C
:105440006B817C818D812DDB0F5FCC0CDD1C0930E5
:1054500001F7F501F292E2921F5F1B3049F60E94BC
:105460004B0D48C080912205843031F180E00E94CC
:10547000A8041092DA0488E190E00FB6F894A89599
:10548000809360000FBE1093600083B7817F8460BB
:1054900083BF83B7816083BF7894889583B78E7FFD
:1054A00083BF0FB6F894A8958091600088618093BF
:1054B0006000109260000FBEA7DDEAE0F5E0819188
:1054C0009191892B09F00AC6A0E2B5E0AE17BF079B
:1054D000B1F780912205853009F4C4CF0E943D11B7
:1054E0000E94320B0E94A80467CF2817390709F0E1
:1054F0007ACF86DBE0900E06F0900F06E114F104FF
:1055000091F18090F7049090F804A090F904B09085
:10551000FA040E944B0D681979098A099B09809049
:10552000F3049090F404A090F504B090F60468158C
:1055300079058A059B05B8F0C7010E94CE1010922C
:105540000F0610920E061092F7041092F8041092B3
:10555000F9041092FA041092F3041092F4041092D9
:10556000F5041092F604C0909606D0909706C114E8
:10557000D10439F1A0909806B09099060E94F40BDE
:105580007C01EA18FB08C6010E9488178E159F054A
:10559000C0F42091960630919706C9019927287F7B
:1055A0003327232B09F07EC174E0880F991F7A9569
:1055B000E1F78A5E994FDC0115962C9122FF0E943B
:1055C0005D1480918D05811569F00E94F40B209186
:1055D0008E0530918F05821B930B8F3F9F4710F4F0
:1055E0000E94341180919D06811509F444C0809178
:1055F0009C06E0919E06E695E695E81BE093FD0487
:10560000853109F4A7C108F05DC1893009F498C15A
:1056100008F04BC1823009F481C1863009F487C19A
:1056200060EDE62E67E0F62E09EA17E08091FE04B1
:10563000811561F01092FE040E94F40B9093FC041B
:105640008093FB04109200051092FF040E94F40B5B
:105650002091FB043091FC04821B930B8F3F9F47EA
:1056600050F42E0D3F1D3093FC042093FB048BEF70
:1056700094E0F801099586E0EDE7F5E0DE0111968A
:1056800001900D928A95E1F790907E05B0907F058C
:10569000F0908005A0908105E090820510927F0532
:1056A0001092800510928105109282058F2D8B2912
:1056B000811509F441C0C0900305D09004050E94F3
:1056C000F40B9C012C193D0990917B05911509F46F
:1056D00000C52531310580F19F3F19F09F5F909300
:1056E0007B05B11459F00E94E80A91E01B140CF0FC
:1056F0009FEF899F802D112480937F05F11459F02D
:105700000E94E80A91E01F140CF09FEF899F802D02
:1057100011248093800580917F05811569F0D090D8
:105720008005D11449F00E94DA0A80937F058D2DFF
:105730000E94DA0A809380058A2D8E29811509F44A
:1057400041C0C0900105D09002050E94F40B9C015D
:105750002C193D0990917A05911509F4B5C42135AC
:10576000310580F19F3F19F09F5F90937A05A11456
:1057700059F00E94080B91E01A140CF09FEF899FDA
:10578000802D112480938105E11459F00E94080BAB
:1057900091E01E140CF09FEF899F802D11248093BF
:1057A000820580918105811569F0D0908205D11420
:1057B00049F00E94DA0A809381058D2D0E94DA0A51
:1057C0008093820580917E05981219C080917F0593
:1057D000811511F08B1113C020918005211511F056
:1057E0002F110DC090918205911511F09E1107C0E7
:1057F00030918105311103C0822B892B81110E94C8
:10580000670C86E0FE013196ADE7B5E001900D92A0
:105810008A95E1F70E94320BF82E80910505F81663
:1058200039F0F09205050E944B0D8F2D0E94A804BF
:1058300080912205843009F0B9CD83E08093E9009E
:105840008091E80082FFB2CD8091E80090E085FF72
:1058500006C00E94100E811509F485C091E0809168
:10586000E8008B778093E800911509F49FCDE090D4
:105870002505F0902605E981E114F10409F492C0B0
:10588000EE3F09F0B2C08A81833020F0855083302A
:1058900008F0ABC0EA81EE3008F0A7C0F0E0E059B4
:1058A000FB4CF7C580E090E086CE8F3009F0B8CE93
:1058B000E695F0E0E854F94FE491EE2EF12C0EEF6E
:1058C00018E0B4CE54EFE52EFF24F3940AE21AE078
:1058D000843209F4ABCE90F448E2E42EF12C06EACF
:1058E00019E0883109F4A2CE833209F099CEE3EBB6
:1058F000F6E0E590F59006E818E098CE853209F0DC
:105900008FCE8E2F63E085D5E92FF0E0E055F94F7B
:10591000E491EE2EF12C03E018E188CEF0E0EF5395
:10592000F94FE491EE2EF12C03EC18E07FCEF0E07D
:10593000E254F94FE491EE2EF12C04EB18E076CE10
:10594000E695F0E0E554F94FE491EE2EF12C06EDEA
:1059500018E06CCEF0E0EB54F94FE491EE2EF12C10
:105960000BE519E063CE30E2C32ED12C9E012F5FF0
:105970003F4F79018091E80085FD0AC08091E800E1
:105980008B778093E8000E94100E811599F366CF03
:105990008091F100D7018D937D01B1E0CB1AD10840
:1059A00049F75CCFE43148F4E11551F0E150E331BF
:1059B00038F4F0E0E258FB4C6CC5EE3F09F46ACFD6
:1059C0008FEF898312C01A8289E08B830EC08A818F
:1059D000823081F08330B1F0813091F70E944B0D1D
:1059E0005ED56B837C838D839E83CE0101960E945E
:1059F000600EDCCC88E290E061D61B821C821D82A6
:105A00008E83F3CF8091200590912105892B69F336
:105A1000FE013196D2018C9111969C91B2E04B0E11
:105A2000511C92838383329620E2421625E052066F
:105A300089F7DBCF8A81823019F66B817C818D8179
:105A40009E812DD588E290E05AD6CFCF4C816B81D4
:105A50008A810E94DD149827892798279E838D8349
:105A6000C4CF2D813E813227232732274C816B8181
:105A70008A810E94DF0FB9CF0E947816B6CF8A8143
:105A8000823891F1B0F48038E9F0813809F0ADCF77
:105A900060E08B810E948C199B8180919E06911100
:105AA0001AC08E7F80939E0610929D060E94540815
:105AB0009CCF833809F099CF20E04091A1066C81FA
:105AC0008B8106C020E04B816091A00680919F06EB
:105AD0000E94D9188ACF816080939E0660E08695E7
:105AE00086950E948C1981CF8B818093A2067DCFF1
:105AF0008A818238E1F060F48038A1F0813809F0C1
:105B000074CF80919E0680FF10C0869586955DCFEC
:105B1000833809F06ACF80919F068B838091A0061D
:105B20008C8363CF8091A10650CF80E04ECF8091CF
:105B3000A2064BCF0E943F088EE996E00E9498187B
:105B400054CF80E18A8351CF1A8285EE3ECF8C817B
:105B50008D3108F04ACF8A809B809824892498242C
:105B6000A12CB12C8E010F5F1F4F7801E80EF11CA4
:105B7000E016F10609F439CF80E035EE8316910482
:105B8000A104B10420F4C401855E9C4F97D5D801CF
:105B900014968C930F5F1F4FBFEF8B1A9B0AAB0AB3
:105BA000BB0AE6CF8091200590912105892B09F44D
:105BB0001CCF8C818D3108F018CF882E912CA12C10
:105BC000B12CCA80DB80DC24CD24DC24E12CF12C38
:105BD0008E010F5F1F4F412C512C32014814590484
:105BE0006A047B0408F001CFE5EECE16D104E1048F
:105BF000F10438F4D80114966C91C601855E9C4F6F
:105C00007ED5BFEF4B1A5B0A6B0A7B0AEFEFCE1A09
:105C1000DE0AEE0AFE0A0F5F1F4FE0CF53D9E5CE32
:105C200083E090CF8C818D3108F0DFCE882E912CCF
:105C3000A12CB12CCA80DB80DC24CD24DC24E12C17
:105C4000F12C412C512C32018E010B5F1F4F481457
:105C500059046A047B0408F0C8CE80E0F2E5CF1650
:105C6000F2E0DF06E104F10418F4C601899626D5B6
:105C7000D8018D938D01BFEF4B1A5B0A6B0A7B0A2B
:105C8000EFEFCE1ADE0AEE0AFE0AE1CF2C81022FD8
:105C900010E02D3108F0A9CE8A819B8198278927B1
:105CA00098272C01612C712C8235F2E09F0708F0B7
:105CB0009CCE822E912CA12CB12C42E552E060E0CA
:105CC00070E04419550966097709421751056105C5
:105CD000710508F48ACE2091200530912105232BEF
:105CE00009F03EC01C0129E2220E311C80FBEE248B
:105CF000FF24E0F880FF0BC08896E0D49D818927BF
:105D00009827892781159C4711F48FEF8D83D50142
:105D1000C401840D951DA61DB71D80FF19C0680123
:105D200041E0C41AD108CE0105968C0D9D1D9CA79B
:105D30008BA7C101800F911FC1D4ABA5BCA59C91BD
:105D400081159C4721F48FEFEBA5FCA5808386018C
:105D5000FE013196EE0DFF1D2FEFE016F10638F033
:105D60008E010F5F1F4FC12CD12C760125C094816D
:105D7000858181159C4711F42483258342E0E40E3C
:105D8000F11C3296EACF82E5481682E0580661049B
:105D9000710430F4D80114966C91C2018996AFD485
:105DA000BFEFCB1ADB0AEB0AFB0AEFEF4E1A5E0AD3
:105DB0006E0A7E0A0F5F1F4FC814D904EA04FB0461
:105DC00010F313CE8091200590912105892B09F4C1
:105DD0000CCECE0101960E94600EFFEF21EE34E062
:105DE000F15020403040E1F700C00000A9CA88E02F
:105DF000E3E2F1E0DE01919601900D928A95E1F7E0
:105E0000FE0132968FE1DF011D928A95E9F786E067
:105E1000898388E07F96DE01159601900D928A9520
:105E2000E1F7E3CD8CE8898381E08A831B821C82C1
:105E3000DCCD8B819C81092E000CAA0BBB0B25E0CD
:105E4000880F991FAA1FBB1F2A95D1F7AC01BD016E
:105E5000405E5F4F6F4F7F4F481759076A077B07B8
:105E600008F4C3CD8C38E1E09E07A105B10508F028
:105E7000BCCD4D38F1E05F076105710520F04CE8BD
:105E800051E060E070E0481B590BBC016B53794F47
:105E9000CE010196D9D3A9CD4AE150E06FEF70E071
:105EA000CE010796F4D3809120058983EA821B8274
:105EB0001C8286E08D8383E0A3CD81E090E0909307
:105EC00026058093250582E390E090930905809351
:105ED00008050E94F40B909307058093060585CD75
:105EE000E114F10481F1D0900A05C09016050091EB
:105EF0000605109107050E94F40B801B910B853657
:105F0000910540F1C3FE26C0D0FE24C00E94F40BD0
:105F100090930705809306058091080590910905E7
:105F200001979093090580930805892B61F41092DD
:105F300026051092250581E090E09093210580933D
:105F40002005E12CF12C809120058983EA82809143
:105F500008053BCD82E390E0909309058093080506
:105F6000F2CF10922105109220053FCD40E250E083
:105F70006FEF70E0CE0101968AD337CD8B818230EE
:105F800009F450C078F4811136C0FE0132968EE1DA
:105F9000DF011D928A95E9F788E089838B8383E08E
:105FA00088A323CD853009F472C0863009F01DCD59
:105FB0001C818AE0FE013596DE01919601900D92DA
:105FC0008A95E1F78BA19CA10E94600A9CA38BA3F8
:105FD0008FEF183060F4FAE01F9FB0011124655371
:105FE0007D4F4AE050E0CE018196A7D380E08983BF
:105FF0000E94F416FACC8C819AE0F92E8E010F5D86
:106000001F4FF8012F2D11922A95E9F7B8010E9430
:1060100073178983F801DE01129601900D92FA94AC
:10602000E1F7E3CC1C818AE0FE013596DE01919612
:1060300001900D928A95E1F789A19AA10E94600AC8
:106040009AA389A38BA19CA10E94600A9CA38BA305
:106050008DA19EA10E94600A9EA38DA38FA198A5E9
:106060000E94600A98A78FA38FEF183060F43AE07F
:10607000139FB001112465587D4F4AE050E0CE01D6
:1060800081965BD380E089830E946D0AAECC2C811F
:106090006AE0CE018196DC01E62F1D92EA95E9F7D0
:1060A000283080F4629FB001112465537D4F4AE08F
:1060B00050E0F4D280E089838AE0FE01B196DE01EF
:1060C0001296ABCE8FEFF7CF2B30310508F04CCBCB
:1060D00079CB2B30310508F001CB2ECB8091DB043E
:1060E000811509F4F6C9B0E1B9BDE2E1E9BD09B431
:1060F00000FEFDCF8091D8008F7D8093D8008091E5
:10610000E00082608093E0008091E00081FDFCCFA0
:106110000E943D11DEC91F921FB61F9211248F935A
:106120009F93AF93BF938091DA04811113C0809144
:10613000280290912902A0912A02B0912B02419647
:10614000A11DB11D8093280290932902A0932A02D9
:10615000B0932B02BF91AF919F918F911F901FBE63
:106160001F90189578941F921FB61F9211248F9339
:106170009F93AF93BF938091280290912902A091A1
:106180002A02B0912B020196A11DB11D8093280215
:1061900090932902A0932A02B0932B02BF91AF9152
:1061A0009F918F911F901FBE1F9018951F920F9265
:1061B0000FB60F9211242F933F934F935F936F93DA
:1061C0007F938F939F93AF93BF93EF93FF938091B0
:1061D000E10082FF09C08091E20082FF05C080914A
:1061E000E1008B7F8093E1008091DA0080FF24C082
:1061F0008091D80080FF20C08091DA008E7F80934C
:10620000DA008091D90080FFA9C080E189BD82E1D8
:1062100089BD09B400FEFDCF81E080932205809105
:106220001702811109C00E94410E0E949E0E8091AA
:10623000E20084608093E2008091E10080FF1AC058
:106240008091E20080FF16C08091E2008E7F8093F3
:10625000E2008091E20080618093E2008091D800AA
:1062600080628093D80019BC85E08093220583E08A
:10627000809321018091E10084FF2FC08091E20092
:1062800084FF2BC080E189BD82E189BD09B400FE95
:10629000FDCF8091D8008F7D8093D8008091E10060
:1062A0008F7E8093E1008091E2008F7E8093E200F8
:1062B0008091E20081608093E20080911602811556
:1062C00009F452C084E08093220580912205843035
:1062D00009F052C082E0809321018091E10083FFA8
:1062E0002CC08091E20083FF28C08091E100877F6D
:1062F0008093E10082E08093220510921602809143
:10630000E1008E7F8093E1008091E2008E7F809398
:10631000E2008091E20080618093E20042E060E070
:1063200080E00E946E0E8091F00088608093F00003
:1063300081E08093210180932001FF91EF91BF9133
:10634000AF919F918F917F916F915F914F913F910D
:106350002F910F900FBE0F901F90189519BC10929F
:1063600022051092170268CF8091E30087FF02C0D8
:1063700083E0A9CF81E0A7CF81E0ADCF1F920F923C
:106380000FB60F921124EF92FF920F931F932F934A
:106390003F934F935F936F937F938F939F93AF93AD
:1063A000BF93CF93EF93FF9309EE10E0F801808144
:1063B000C091EC008F70C795CC27C795C82B108271
:1063C00080EFE82EF12CF7018081877F808378941D
:1063D0000E947E11F8011082F7018081886080831D
:1063E000CF70F801C083FF91EF91CF91BF91AF9132
:1063F0009F918F917F916F915F914F913F912F91DD
:106400001F910F91FF90EF900F900FBE0F901F9074
:106410001895992778E0880F991F961708F0961B12
:10642000881F7A95C9F78095089587FB082E062660
:1064300087FD819567FD6195ECDF0EF4919507FC72
:1064400081950895AA1BBB1B51E107C0AA1FBB1F62
:10645000A617B70710F0A61BB70B881F991F5A95F0
:10646000A9F780959095BC01CD01089597FB072E63
:1064700016F4009406D077FD08D0E4DF07FC05D0C1
:106480003EF4909581959F4F0895709561957F4F4B
:106490000895EE0FFF1F0590F491E02D09946927F0
:1064A000962769277827872778270895ABD1332344
:1064B00012F48A1B9B0B01C0A5D1B7FF0895821B64
:1064C000930B08952F923F924F925F926F927F921B
:1064D0008F929F92AF92BF92CF92DF92EF92FF92F4
:1064E0000F931F93CF93DF93CDB7DEB7CA1BDB0BA0
:1064F0000FB6F894DEBF0FBECDBF09942A88398845
:1065000048885F846E847D848C849B84AA84B9844B
:10651000C884DF80EE80FD800C811B81AA81B98157
:10652000CE0FD11D0FB6F894DEBF0FBECDBFED016B
:106530000895002E083090F0982F872F762F652F22
:10654000542F432F322F22270850F4CF220F331F0E
:10655000441F551F661F771F881F991F0A95B2F7A2
:10656000002D089597FD1094002E083098F00850E3
:10657000232F342F452F562F672F782F892F912DBA
:10658000F4CF159497958795779567955795479587
:10659000379527950A95AAF71124002D08958F9213
:1065A0009F92AF92BF92CF92DF92EF92FF92CF93E2
:1065B000DF93EC01688179818A819B816115710586
:1065C0008105910521F464E279ED8BE597E02DE1F9
:1065D00033EF41E050E0C8D049015A019B01AC01C2
:1065E000A7EAB1E4DDD06B017C01ACEEB4EFA5010C
:1065F0009401E2D0DC01CB018C0D9D1DAE1DBF1DB1
:10660000B7FF03C00197A109B04888839983AA8383
:10661000BB839F77DF91CF91FF90EF90DF90CF907A
:10662000BF90AF909F908F900895B9CF80E091E098
:10663000B6CFA0E0B0E08093000190930101A09359
:106640000201B09303010895FB01DC0102C0059033
:106650000D9241505040D8F70895FC0141505040F0
:1066600030F001900616D1F73197CF0108958827B1
:1066700099270895FB01DC0104C08D9101908019D8
:1066800021F441505040C8F7881B990B0895DC0154
:1066900001C06D9341505040E0F70895DC01CB01FB
:1066A000FC01F999FECF06C0F2BDE1BDF89A319622
:1066B00000B40D9241505040B8F70895F999FECFBB
:1066C00092BD81BDF89A992780B50895A6E1B0E002
:1066D00044E050E0E5CFA8E1B0E042E050E0E0CF98
:1066E000DC01A40FB51F4150504040F0CB01840F96
:1066F000951F2E9105D041505040D8F70895262F70
:10670000F999FECF92BD81BDF89A019700B40216A7
:1067100039F01FBA20BD0FB6F894FA9AF99A0FBE55
:1067200008950396272FECDFEADF252FE9DF242FDA
:10673000E7CF0196272FE4DFE2CFDC01CB0102C0D7
:106740002D9105D041505040D8F70895262FF99942
:10675000FECF1FBA92BD81BD20BD0FB6F894FA9A44
:10676000F99A0FBE01960895052E97FB16F4009432
:106770000FD057FD05D024D007FC02D046F408C046
:1067800050954095309521953F4F4F4F5F4F08955D
:1067900090958095709561957F4F8F4F9F4F08958D
:1067A00031D0A59F900DB49F900DA49F800D911D99
:1067B00011240895B7FFF4CFF3DF821B930B0895E4
:1067C000A1E21A2EAA1BBB1BFD010DC0AA1FBB1FF5
:1067D000EE1FFF1FA217B307E407F50720F0A21B67
:1067E000B30BE40BF50B661F771F881F991F1A94D4
:1067F00069F760957095809590959B01AC01BD01FE
:10680000CF010895A29FB001B39FC001A39F700D57
:10681000811D1124911DB29F700D811D1124911DA8
:106820000895F894FFCF9C0CA10CA30CA80CB80CF5
:10683000B80CB80CB80CB80CB80CB80CB80CAA0C46
:10684000AE0CB10CB60CC60CCC0CD00C5B12811289
:10685000871281128712D912FA12871200140D14AE
:106860002C1F941F341FFE1E021F381F061F3C1FC3
:10687000481F121F8D1F161F4C1F1A1F501F751FF8
:106880001E1F541F7C1F241F5A1F621F0A1F401FF8
:106890000E1F441F281F5E1F6C1F851F8B1FF81EB5
:1068A000301F9B1FCA1ED01EBD1EC41ED61EDC1E5E
:1068B000E21EBB1FD21FD61FDA1FDE1FE21FE61F1C
:1068C000EA1FEE1FF21FF61F482148217F217F217A
:1068D0002F224A22A321A3214F22C422D522D5222E
:1068E000F72E122F192FF52CF52C4C2F5D2F702F12
:1068F000B12FB62FF52CF52CF52CBE2FE32CE72C61
:106900001A2D262D312D3C2D3F2D782D9A2DE02C42
:10691000E22EA12DA42DA72DD22D0E2E102E122E3B
:02692000462E01
:106922000100000001010201191A1B1C1D1E1F207B
:106932002122F10BA30FB90FBE0FC30F9A0F000054
:10694200010001F40E0077A2555A3E4422B684019A
:106952006201AC008A02A302C30200010202020227
:106962000606060909090909090F0F0F0F0F0F156E
:10697200151518191919191919191919192324256D
:106982002525252525909192939594969734C63086
:1069920031323337F7F6F5F4F1E200E900EA00B5F7
:1069A20000B600B700CD008301CC008A01920194A9
:1069B200012102230224022502260227022A02B30F
:1069C20000B4006F0070009F01CB019F02A002E2A1
:1069D20000E900EA00B500B600B700CD008301CCA3
:1069E200008A019201940121022302240225022637
:1069F2000227022A02B300B4006F0070009F01CB8D
:066A0200019F02A002004A
:00000001FF
